:020000040000fa
:080000000002040000000000f2
:020000040000fa
:100008006203000062030000620300006203000054
:100018006203000062030000620300006203000044
:100028006203000062030000620300005242000005
:10003800620300006203000062030000f85c000035
:10004800620300006203000062030000d2020000a5
:100058000003000062030000620300006203000066
:1000680062030000620300006203000062030000f4
:1000780062030000620300006203000062030000e4
:1000880062030000620300006203000062030000d4
:1000980062030000620300006203000062030000c4
:1000a80062030000620300006203000062030000b4
:1000b80062030000620300006203000062030000a4
:1000c8006203000062030000620300006203000094
:1000d8006203000062030000620300006203000084
:1000e8006203000062030000620300006203000074
:1000f8006203000062030000620300006203000064
:100108006203000062030000620300006203000053
:100118006203000062030000620300006203000043
:100128006203000062030000620300006203000033
:100138006203000062030000620300006203000023
:100148006203000062030000620300006203000013
:100158006203000062030000620300006203000003
:1001680062030000620300006203000062030000f3
:1001780062030000620300006203000062030000e3
:1001880062030000620300006203000062030000d3
:1001980062030000620300006203000062030000c3
:1001a80062030000620300006203000062030000b3
:1001b800245b000062030000620300006203000089
:1001c8006203000062030000620300006203000093
:1001d8006203000062030000620300006203000083
:1001e8006203000062030000620300006203000073
:0801f800620300006203000035
:020000040000fa
:100208006203000062030000620300006203000052
:100218006203000062030000620300006203000042
:100228006203000062030000620300005242000003
:10023800620300006203000062030000f85c000033
:10024800620300006203000062030000d2020000a3
:100258000003000062030000620300006203000064
:1002680062030000620300006203000062030000f2
:1002780062030000620300006203000062030000e2
:1002880062030000620300006203000062030000d2
:1002980062030000620300006203000062030000c2
:1002a80062030000620300006203000062030000b2
:1002b80062030000620300006203000062030000a2
:1002c8006203000062030000620300006203000092
:1002d8006203000062030000620300006203000082
:1002e8006203000062030000620300006203000072
:1002f8006203000062030000620300006203000062
:100308006203000062030000620300006203000051
:100318006203000062030000620300006203000041
:100328006203000062030000620300006203000031
:100338006203000062030000620300006203000021
:100348006203000062030000620300006203000011
:100358006203000062030000620300006203000001
:1003680062030000620300006203000062030000f1
:1003780062030000620300006203000062030000e1
:1003880062030000620300006203000062030000d1
:1003980062030000620300006203000062030000c1
:1003a80062030000620300006203000062030000b1
:1003b800245b000062030000620300006203000087
:1003c8006203000062030000620300006203000091
:1003d8006203000062030000620300006203000081
:1003e8006203000062030000620300006203000071
:0803f800620300006203000033
:020000040000fa
:10040000afcc2000ce2925000e018800000000009e
:10041000000020000000e000020032000001200087
:10042000200288000c00070060402400010020002a
:100430000f000700000020000000e0000200320072
:1004400000000200000000009c43020000000000c9
:100450000040da000000fe00a06b20000000e00079
:1004600002003200002020009001880000000600f9
:10047000a1028800800078000000eb001a0037001d
:10048000e280400054a0b4009101ba00e280400034
:1004900054a0b4009102ba00e280400054a0b4001d
:1004a0000002eb00472bde00f507b200a601880032
:1004b000602ce10008003a000049eb000201e8006e
:1004c000020039003420ec0002f0a0008301e900b2
:1004d000f9ff3e00040037006128e100010032000e
:1004e0000082eb00040007001101ba000200e000e6
:1004f000e3ff3a000000060004d0a300e20f490029
:100500001c003900810278003549ba000201e80078
:10051000020039003420ec0002f0a0008301e90061
:100520000f0032002549ba000201e800020039003c
:100530003420ec0002f0a0008301e9000800320042
:100540000400e0000600320015c9ba000201e8000c
:10055000020039003420ec0002f0a0008301e90021
:100560008180e80054a0b4000300e000e2ff3a00fc
:10057000000006009102ba00055978008301e900e5
:10058000f7ff3200c82ade00055978008301e90030
:10059000f3ff32000400e000f1ff320011d9ba008d
:1005a000eeff3700841f78000200fa008560a90082
:1005b0001411800062026200e00f5200020032005b
:1005c0002222a9000b00370014118000640262008f
:1005d000e00f520007003a0002003700341180009b
:1005e000044f78001411800061026200e00f520095
:1005f000faff3a000080fa004f027800004006003f
:10060000841f78000200fa0004488000040f78007c
:100610001e027800241188008580a9000080fa005d
:100620004f027800004006000000fa0042c7a9000f
:100630002535800004fc2f00048262007400b300a2
:10064000243588003536800004fc2f0004826200c7
:100650003400b3003436880042c7a800f4192000e3
:10066000441188000002eb00041188002062a800f9
:100670000002eb001411880021e2a8002342a80028
:100680008560a9009560a800950580000470200091
:1006900005027200940588000080fa000000060040
:1006a0000400fa00000f7800110798001e0278007d
:1006b000044888000002eb00040078000080fa0083
:1006c000000006000040da000000fe0003f0a20077
:1006d000889fbe008a9fbe008c1f78000001070023
:1006e000070133006450e1004f0032006420e10054
:1006f0005200320003826c0007003b000905d00065
:100700000306d000820f54000c065d000200390081
:1007100002003200890178000306780085825500c6
:1007200004003d000003fd008103fd008502ea0096
:100730008b854200840f720002003b0060001000b5
:10074000e08018006011b8000005eb007a28e10095
:100750000a00390006007800c75ddd00f707b20027
:10076000878075002d003700828171000a017800b2
:10077000610560008180d1000080d3008502e9001e
:10078000f9ff3b00060440008784480002003b005c
:1007900060041400e0841c000988a30007003200f4
:1007a0008a81710082817100610164008904d10035
:1007b0000884d3008b05e800170037000978a300f0
:1007c00013003a000b00e000130034008b05e90031
:1007d0000804440089844c000a4474000978a3008a
:1007e0000d003a000b00e000070034008b05e90023
:1007f0000804440089844c0001003a000b002000ea
:100800000978a300f7ff32000001eb000200370077
:10081000828171000a017800760007000cf0a700c1
:1008200001f0a000bf0037006420e10002003a00a0
:10083000838f6c00bf0033000801be000200be00c1
:10084000b80037000081eb00f1003700889fbe0040
:100850008a9fbe008c1f7800a1000700a80033000b
:1008600003866c006450e1002e0032006420e10039
:10087000330032006150e1002f0032006120e100be
:100880003100320085855500eb07b00009002000db
:1008900008042000050037000804440089844c0047
:1008a0000a0031000603430087834b000001530018
:1008b00081815b00f8ff33000203be000800a00046
:1008c0000804440089844c00f6ff3900c639dd0075
:1008d0008301730001003200130020008904d1005d
:1008e0000884d3000998a300050032000800a7007f
:1008f0000300a0008904d1000884d3008b05e80020
:100900008904d1000884d3000001eb000281d200e9
:100910003800070001f0a1000cf0a70001f0a000d2
:10092000800037006420e100820032000801be0030
:100930000200be00f7ff37006120e1007d003200b9
:100940006000b800f3ff37000000200001f8270026
:10095000f0ff3700f4ff2f001b0137000001be003d
:100960004a0007000470a70003f0a1006509b10068
:10097000160032000d0035006828e1000600350041
:10098000f0ff2f00f1ff27000300e00013003b0001
:1009900001002800000005000000400081804800a0
:1009a0008502e900fcff3a0008003700f88f42009a
:1009b00002003c008000eb00000005008100d10037
:1009c0000080d3008502e800fcff3a000300e0004d
:1009d00002003b0060001000e080180000000600ec
:1009e0004f89de0082017800140137006011b800e1
:1009f0002201370081002000618055000b003d007e
:100a00000b00200061fe2f000100e1001d003400fa
:100a100082817100610164008904d1000884d300df
:100a20000000e800faff3a00710020006100640055
:100a300003007000020060000900320061044400fd
:100a4000e0844c000988a500050032008b05e80011
:100a50006808e10002003a008904d1000884d3004c
:100a6000f20f20000258e10005003d00c75ddd00e7
:100a7000f907b200898075000800780000000600c0
:100a80000bf827008b00780000000500c70ade0085
:100a9000f107b200f50fb20008003200e1cf4200ca
:100aa000020032000170a00024000500810f7000d8
:100ab000010032000408050044000500810f7000a9
:100ac00002003a00140005008502e9000000400021
:100ad00081c04800fcff3b000170a000240005001d
:100ae0000004be00e9ff07000003be000405be00cd
:100af0000200be00e5ff0700844f750000000600fd
:100b00000200be006450e100050036006420e100f0
:100b1000020036000968a30001003a000800be0088
:100b20000160a0004f0678004f05be004f04be00d4
:100b300000000600f0ff2f00f1ff2700f9ff37004b
:100b4000889fbe008a9fbe008c1f7800e4ff0700cc
:100b5000ebff330003866c006450e1002400320098
:100b60006420e100270032006150e10022003200e1
:100b70006120e100210032008b854200eb07b100cb
:100b80000134b800003ab8000804420089844a00e1
:100b9000013ab8000030b8008880400009014a00de
:100ba0000400330000004000818048000201490039
:100bb0008b05e900c909dd008301700001003200e6
:100bc00013002000c814de004814dd004709de00d1
:100bd0001200b200c808de000884700085ff07001c
:100be00001f0a1000cf0a70001f0a000cdff37003c
:100bf0006120e100cfff32000801be000200be000c
:100c0000f7ff37006150e100fcff3a00c9ff3700f1
:100c1000889fbe008a9fbe008c9fbe008205780020
:100c20000004be0099ff07000800be006420e10038
:100c30000700390002003a00f1ff2700f0ff2f0003
:100c40000160a000120220001266880055003700e3
:100c50006120e10003003a000b00a70001f8230027
:100c60005000370001f0a10002002100936424002d
:100c7000700007000800be0004003500b2fd20002f
:100c8000930c2400ac0007000004be000005eb003c
:100c90000b00a6004f0dde0001f0a1000004be0015
:100ca00032982f0023ea2300a5ff07000001eb0084
:100cb00003f023000b00a70003f8230084fe0700c5
:100cc00026ff07000000a7000a00a20044ff07005b
:100cd0000b00e000030032000200200003f02300bc
:100ce0007afe070001f0a2000006be00020020000c
:100cf0009304240092ff07000801be0074fe070061
:100d0000809fbe000c00be0022a22a00d3a72300b1
:100d10008bff07004f01be006dfe07000004be0000
:100d200001f0a10002002000039823004100070009
:100d30000800be00190035000001be0080ff07005a
:100d40000006be00b2c52900e36223007cff070055
:100d500022222b00f3942b005dfe07000c01be0045
:100d600077ff0700e273280083c0230058fe0700c6
:100d70000c01be0072ff070042aa2a00a3e22b006a
:100d800053fe07000c01be006dff07000801be0006
:100d90006bff07000801be004dfe07000a00a70018
:100da00001f0a2004f06be004f05be004f04be007a
:100db000000006000001eb0095ff3700af000700c0
:100dc0000400be0000000600889fbe008a9fbe008f
:100dd000841f780042ff07004f00780011003300a5
:100de000f0ff2f00838f6c0006003b0004056500b8
:100df0000a00a7000800370009f0a6001000200034
:100e000008003700820f5400838f5c000300390014
:100e10001000200001003e000000200009f0a700a3
:100e20000000ea004f05be004f04be000000e000d5
:100e30000000060014002000e3ff3700881f780040
:100e4000030478000300e00007003d00600010008c
:100e5000e080180060011900e081190002003b00e9
:100e600001f02d00030037000400070008f0a70080
:100e700001f0a0004f04780000000600889fbe002b
:100e80008a9fbe000082700004027100048271001b
:100e9000260032000004be000200be006011b8004f
:100ea0006b092000950220000182cf000a00390062
:100eb0000541b1000082cf00070039000541b100b3
:100ec0000982cf00040039000541b1000882cf003b
:100ed000010039000541b100054252001200320004
:100ee0000a003b0082817100610164008100d10031
:100ef0000080d3008984d3000884d3008b05e800e8
:100f00000442e800f7ff3a000700370008044400f5
:100f100089844c0000004800818048008b05e9006e
:100f20000442e900f9ff3a00b2fe07004f05be0097
:100f30004f04be000000060004002000000037003f
:100f4000889fbe008a9fbe008c1f78004f26dd0060
:100f5000e3fe0700eafe33006120e10043003200b7
:100f60006250e10041003e003e0039006420e10093
:100f70003c003200058255000f003b000402e800ef
:100f800038003a00800f5300818f5b003500340039
:100f90000800be0003f0a10001f0a60003f0a000cd
:100fa0000cf0a700cafd0700defe37000603430071
:100fb00087834b000c4646000005530081855b008b
:100fc000020033000a03be000c00a0000402e90086
:100fd000f6ff3b00850578000602430087824b0040
:100fe00004003a006000b80009f0a70001f0a0007a
:100ff000ccfe37000002520081825a000704e00054
:10100000040033000603430087834b008b05e9008f
:10101000faff3700090578000604be000203be008f
:101020006011b80073fe0700e00f5200e08f5a0015
:101030000700350002003c000c08a3000400320049
:101040000601be0003f0a0000cf0a700a0fd070001
:101050000a85680001f0a1000af0a70001f0a000d5
:10106000b0fe37000800be00aefe370010022000c0
:101070000cf0a60010668800aefe37006022b800b3
:10108000060220000000d0008180d2000482d2003d
:101090008582d2000000a0000202520083825a0022
:1010a000030031000202420083824a000000a100d6
:1010b0000603e900f3ff3a000000060015c0b30084
:1010c0000100200084cc2000206688003166880062
:1010d000054a78000000060084cc20008042eb0026
:1010e00094cf120002003a0010002000f3ff070026
:1010f0002066800031668000d2e62400631c240054
:101100002400070094032300050020000002420091
:1011100081824a00246688003566880005007800d0
:1011200000f0a100000006000002eb008002780041
:101130000500370061437a0061015100e0815900e8
:1011400086727a000402e800e00f5100e08f590037
:10115000f8ff3a0000000600000278000000eb00f3
:101160000401e80084027800030020006103b80055
:101170000000e8008600410065437b00e04f53001b
:10118000faff3a000482ea0004804000cf80de00cb
:1011900000000600020ab900001bb9000200b800f6
:0c11a000810042008100430000000600b6
:020000040000fa
:1011ac00000000000000000001010000010200002e
:1011bc0002030000040500000506000007090000fa
:1011cc000a0b00000c0e00000f110000121400009e
:1011dc0015170000191b00001d1f00002123000023
:1011ec00252800002a2c00002f3100003436000086
:1011fc00393b00003e41000043460000494c0000d2
:10120c004f520000555800005a5d00006164000008
:10121c00676a00006d70000073760000797c000036
:10122c0080830000868900008c8f0000929500005e
:10123c00989b00009ea20000a5a70000aaad00008c
:10124c00b0b30000b6b90000bcbe0000c1c40000c1
:10125c00c6c90000cbce0000d0d30000d5d700000b
:10126c00dadc0000dee00000e2e40000e6e800006a
:10127c00eaeb0000edee0000f0f10000f3f40000ea
:10128c00f5f60000f8f90000fafa0000fbfc00008b
:10129c00fdfd0000fefe0000feff0000ffff000051
:1012ac00ffff0000ffff0000fefe0000fefd00003f
:1012bc00fdfc0000fbfa0000faf90000f8f6000053
:1012cc00f5f40000f3f10000f0ee0000edeb00008f
:1012dc00eae80000e6e40000e2e00000dedc0000ea
:1012ec00dad70000d5d30000d0ce0000cbc9000067
:1012fc00c6c40000c1be0000bcb90000b6b30000fb
:10130c00b0ad0000aaa70000a5a200009e9b0000a3
:10131c0098950000928f00008c8900008683000055
:10132c00807c000079760000737000006d6a00000c
:10133c0067640000615d00005a58000055520000bf
:10134c004f4c000049460000434100003e3b00006a
:10135c0039360000343100002f2c00002a28000000
:10136c0025230000211f00001d1b00001917000081
:10137c0015140000121100000f0e00000c0b0000e1
:10138c000a09000007060000050500000403000020
:10139c00020200000101000001000000000000003a
:1013ac00fffe0000fdfc0000fbfa0000f9f8000055
:1013bc00f7f60000f5f40000f3f20000f1f0000085
:1013cc00efee0000eceb0000eae90000e8e70000bb
:1013dc00e6e50000e4e30000e2e10000e0df0000ed
:1013ec00dedd0000dcdb0000dad90000d8d700001d
:1013fc00d6d50000d4d30000d2d10000d0cf00004d
:10140c00cecd0000cccb0000cac90000c7c600007e
:10141c00c5c40000c3c20000c1c00000bfbe0000b4
:10142c00bdbc0000bbba0000b9b80000b7b60000e4
:10143c00b5b40000b3b20000b1b00000afae000014
:10144c00adac0000abaa0000a9a80000a7a6000044
:10145c00a5a30000a2a10000a09f00009e9d00007b
:10146c009c9b00009a9900009897000096950000ac
:10147c009493000092910000908f00008e8d0000dc
:10148c008c8b00008a89000088870000868500000c
:10149c0084830000828100007f02000003040000ae
:1014ac000506000007080000090a00000b0c0000ec
:1014bc000d0e00000f10000011120000131400009c
:1014cc001516000017180000191a00001b1c00004c
:1014dc001d1e00001f2000002122000023240000fc
:1014ec0026270000282900002a2b00002c2d0000a4
:1014fc002e2f000030310000323300003435000054
:10150c0036370000383900003a3b00003c3d000003
:10151c003e3f0000404100004243000044450000b3
:10152c0046470000484a00004b4c00004d4e00005e
:10153c004f5000005152000053540000555600000b
:10154c0057580000595a00005b5c00005d5e0000bb
:10155c005f6000006162000063640000656600006b
:10156c0067680000696a00006b6c00006d6f00001a
:10157c0070710000727300007475000076770000c3
:10158c00787900007a7b00007c7d00007e7f000073
:10159c000001000002030000040500000607000023
:1015ac00080900000a0b00000c0d00000e0f0000d3
:1015bc00101100001314000015160000171800007d
:1015cc00191a00001b1c00001d1e00001f2000002b
:1015dc0021220000232400002526000027280000db
:1015ec00292a00002b2c00002d2e00002f3000008b
:1015fc003132000033340000353600003839000039
:10160c003a3b00003c3d00003e3f000040410000e2
:10161c004243000044450000464700004849000092
:10162c004a4b00004c4d00004e4f00005051000042
:10163c0052530000545500005657000058590000f2
:10164c005a5c00005d5e00005f600000616200009b
:10165c00636400006566000067680000696a00004a
:10166c006b6c00006d6e00006f70000071720000fa
:10167c00737400007576000077780000797a0000aa
:10168c007b7c00007d7e0000808100008283000056
:10169c008485000086870000888900008a8b000002
:1016ac008c8d00008e8f00009091000092930000b2
:1016bc009495000096970000989900009a9b000062
:1016cc009c9d00009e9f0000a0a10000a2a3000012
:1016dc00a5a60000a7a80000a9aa0000abac0000ba
:1016ec00adae0000afb00000b1b20000b3b400006a
:1016fc00b5b60000b7b80000b9ba0000bbbc00001a
:10170c00bdbe0000bfc00000c1c20000c3c40000c9
:10171c00c5c60000c7c90000cacb0000cccd000074
:10172c00cecf0000d0d10000d2d30000d4d5000021
:10173c00d6d70000d8d90000dadb0000dcdd0000d1
:10174c00dedf0000e0e10000e2e30000e4e5000081
:10175c00e6e70000e8e90000eaeb0000ecee000030
:10176c00eff00000f1f20000f3f40000f5f60000d9
:10177c00f7f80000f9fa0000fbfc0000fdfe000089
:10178c00ffff0000ffff0000ffff0000ffff000055
:10179c00ffff0000ffff0000ffff0000ffff000045
:1017ac00ffff0000ffff0000ffff0000ffff000035
:1017bc00ffff0000ffff0000ffff0000ffff000025
:1017cc00ffff0000ffff0000ffff0000ffff000015
:1017dc00ffff0000ffff0000ffff0000ffff000005
:1017ec00ffff0000ffff0000ffff0000ffff0000f5
:1017fc00ffff0000ffff0000ffff0000ffff0000e5
:10180c00ffff0000ffff0000ffff0000ffff0000d4
:10181c00ffff0000ffff0000ffff0000ffff0000c4
:10182c00ffff0000ffff0000ffff0000ffff0000b4
:10183c00ffff0000ffff0000ffff0000ffff0000a4
:10184c00ffff0000ffff0000ffff0000ffff000094
:10185c00ffff0000ffff0000ffff0000ffff000084
:10186c00ffff0000ffff0000ffff0000ffff000074
:10187c00ffff0000ffff0000ff0000000000000061
:10188c00000000000000000000000000000000004c
:10189c00000000000000000000000000000000003c
:1018ac00000000000000000000000000000000002c
:1018bc00000000000000000000000000000000001c
:101aec00ffff0000ff0000000000000000000000ed
:101afc0000000000000000000000000000000000da
:101b0c0000000000000000000000000000000000c9
:101b1c0000000000000000000000000000000000b9
:101b2c0000000000000000000000000000000000a9
:101b3c000000000000000000000000000000000099
:101b4c000000000000000000000000000000000089
:101b5c000000000000000000000000000000000079
:101b6c005031000064750000ddaf0000038d0000f3
:101b7c00b1fe0000d7e30000d88e00008d85000078
:101b8c004cd90000fbf100004bf80000cb4b0000df
:101b9c00f84600002ce700001335000090c7000049
:101bac00d0880000ba700000554f000004520000ad
:101bbc007f8d000082dd0000d82f0000236600001e
:101bcc0083d200009b5600000ef30000f6eb0000e1
:101bdc00a7c7000063380000dfcd0000d1ee000085
:101bec0004fc00000f85000047b80000adbd0000ec
:101bfc00ec8d0000c07000004f3500009108000013
:101c0c00a67d000039430000aac00000a7ae00006a
:101c1c0084130000e4040000448e00009a4e00007f
:101c2c0016e000006a330000313c0000a85f0000a1
:101c3c003cd8000080ea00004d370000c8250000a9
:101c4c00ba9a00002e7700004af00000252300000d
:101c5c0099580000743d00006d7a00003ded0000c5
:101c6c00d4a30000b55b00005bc60000fcb2000012
:101c7c0052130000150a00003f8a00000285000084
:101c8c00ade700008123000055bc00009cf700006c
:101c9c008cbf00000595000052cc0000e60b000044
:101cac004ef6000081d9000096d90000afa30000c9
:101cbc008a910000f7830000e1b90000f3420000b4
:101ccc009f6600001847000064170000f17b0000bd
:101cdc00b3be0000e2a300006dcb0000091e0000a3
:101cec00e5e10000b9530000874f0000df930000ce
:101cfc001fcb000082630000e45600009c380000fb
:101d0c00edd800000a9100000ab4000041cf000099
:101d1c0002440000271d000065340000a45100009f
:101d2c0071410000bfb7000000510000d46c0000ee
:101d3c00bbdb00003cc10000bea500002518000064
:101d4c007de80000a2290000e29800009c6e0000d3
:101d5c004e6f000020730000746f00007269000069
:101d6c00657300002c0000004a75000073740000bd
:101d7c0020720000616900006e6200006f77000045
:101d8c00732c000020000000616e00006420000035
:101d9c0074610000696c0000732e00002e2e000090
:101dac0000480000692e0000204800006f770000fa
:101dbc0020270000626f00007574000000610000b5
:101dcc002071000075690000636b00002073000037
:101ddc00746f0000727900003f000000486500003d
:101dec007861000064650000636900006d610000ab
:101dfc006c200000416c0000696500006e730000ef
:101e0c0000620000792000006a6100006d6900002a
:101e1c00736e0000656d00006f000000492000002b
:101e2c00736800006f7500006c640000206800008f
:101e3c0061760000652000000073000074610000f2
:101e4c007274000065640000207300006f6f000066
:101e5c006e650000722e00000054000068610000e6
:101e6c006e6b000073200000746f000020410000b6
:101e7c00726b00006f2c0000004c000061790000b8
:101e8c00657200004f6e0000652c0000204e0000b3
:101e9c00534c00002c000000626c000064650000d4
:101eac00776f00006c6600002c200000616e000053
:101ebc00642000004d49000054000000492000003f
:101ecc006c6f0000766500002074000068690000eb
:101edc0073200000626f000061720000642100003a
:101eec0000570000686500006e270000732000009a
:101efc0074680000652000006e65000078740000b6
:101f0c00007000006172000074790000213f000035
:041f1c0021000000a0
:020000040000fa
:101f200010100000080300000003000003e400009c
:101f30000303000003e400000303000003030000a8
:101f400003030000030300000303000003e4000098
:101f50000303000003030000e403000003e40000a7
:101f600003f5000003030000030300000303000067
:101f700003030000e4030000e4e4000003030000a6
:101f8000e4030000e40300000303000003f5000085
:101f900003030000e4e40000e4e40000e4030000c4
:101fa000e4030000e4030000030300000303000057
:101fb000e4030000e4e40000e4e40000e4e40000e2
:101fc000e40300000303000003030000e403000037
:101fd000e4e4000003e40000e4e40000f5e40000b1
:101fe000e4030000e4f5000003030000e4e4000063
:101ff000e4e40000f5e40000e4e40000e4f500009f
:10200000e4e40000e4e4000003e4000003e4000072
:10201000e4e40000e4e40000e4f50000e4f500007e
:10202000e4e40000e4e4000003e4000003e4000052
:10203000e4e40000e4f50000e4f50000e4f500004d
:10204000f5e40000e4e4000003e40000e4e4000040
:10205000e4e40000f5e40000f5f50000f5f500000b
:10206000f5f50000e4030000e4e40000e4e400000f
:10207000e4f50000f5f50000f5ff0000f5f50000bf
:10208000e4f50000e4e40000e4030000e4e4000000
:10209000f5f50000f5ff0000f5ff0000f5ff00007a
:1020a000f5f50000e4e40000e4030000e4e40000cf
:1020b000f5f50000ffff0000ffff0000fff5000046
:1020c000f5e40000e4e400000303000003e4000082
:1020d000e4f50000f5ff0000ffff0000fff5000041
:1020e000f5e40000e4e400000303000003e4000062
:1020f000e4e40000f5f50000f5f50000f5e400006b
:10210000e4e40000e4030000030300000303000014
:1021100003e40000e4e40000e4e40000e4e4000080
:102120000303000003030000031000001008000078
:10213000030000000303000003030000030300008a
:102140000303000003e400000303000003e40000b5
:10215000030300000303000003f5000003e4000094
:1021600003030000e40300000303000003e4000095
:102170000303000003030000e4030000e403000085
:1021800003e40000e4030000e40300000303000094
:102190000303000003030000e4030000e403000065
:1021a000e4e40000e4e40000e403000003f50000c0
:1021b000030300000303000003030000e4e4000045
:1021c000e4e40000e4e40000e4030000e4030000b1
:1021d0000303000003f50000e4030000e4e4000052
:1021e000f5e40000e4e4000003e40000e403000080
:1021f000e403000003e40000e4e40000e4f5000070
:10220000e4e40000e4e40000f5e40000e4e400009d
:10221000e403000003e40000e4e40000e4f500004f
:10222000e4f50000e4e40000e4e40000e4e400007d
:1022300003e4000003e40000e4e40000f5f500001e
:10224000e4f50000e4f50000e4e40000e4e400004c
:1022500003e40000e4030000e4f50000f5f50000ed
:10226000f5f50000f5e40000f5e40000e4e400000a
:10227000e4e40000e4e40000e4f50000e4f500001c
:10228000f5ff0000f5f50000f5f50000e4e40000be
:10229000e4e40000e4e40000e4f50000f5ff0000e1
:1022a000f5ff0000f5ff0000f5f50000f5e4000083
:1022b000e403000003e40000e4e40000f5f500009e
:1022c000ffff0000ffff0000fff50000f5e4000045
:1022d000e403000003e40000e4e40000f5f500007e
:1022e000ffff0000ffff0000f5f50000e4e4000040
:1022f0000303000003030000e4e40000e4e4000042
:10230000f5f50000f5f50000f5e40000e4e4000058
:1023100003030000030300000303000003e40000c4
:10232000e4e40000e4e40000e4e40000030300004f
:102330000303000008080000080300000003000079
:10234000e4030000e40300000303000003030000b3
:102350000303000003e40000030300000303000084
:1023600003030000e4e40000e403000003030000b2
:10237000e4e40000e4e40000f5e40000e4e400002c
:10238000e4e40000f5f50000f5e40000e4e40000fa
:10239000e4f50000f5ff0000f5f50000e40300009f
:1023a000e4f50000ffff0000f5e40000e403000096
:1023b000e4e40000f5f50000e4e400000308000098
:1023c00008080000030000000303000003030000ee
:1023d000030300000303000003e40000e403000023
:1023e000e4e400000303000003030000e4e4000051
:1023f000e4e40000e403000003e40000e4e400007f
:10240000e4f50000e4e4000003e40000f5e400006b
:10241000e4e40000e4030000e4e40000e4f500006c
:10242000f5f50000e4e4000003e40000f5ff00001f
:10243000ffff0000f5e4000003e40000e4f5000005
:10244000f5f50000e40300003120000008ff000063
:1024500000ff0000ffff0000ffff0000ffff000083
:10246000ffff0000ffff0000ffff0000ffff000074
:10247000ffff0000ffff0000ffff0000ffff000064
:10248000ffff0000ffff0000ffff0000ffff000054
:10249000ffff0000ffff0000ffff0000ffff000044
:1024a000ffff0000ffff0000ffff0000ffff000034
:1024b000ffff0000e0ff0000ffe00000ffff000062
:1024c000e0e00000e0e00000ffff0000e0ff0000af
:1024d000e0e50000ffff0000d8d80000d8ff0000b2
:1024e000ff1d00001d1d00001dff00001d1d000040
:1024f0001d1d00001d2700002727000027ff0000ea
:1025000027c30000ffc30000c3ff0000ffe5000079
:10251000ffff0000ffe0000000ff0000e0000000ff
:10252000e0ff000000000000e0000000ffe000000d
:10253000e0ff000000d80000ffd80000000000000d
:10254000d81d0000ff000000000000001dff00007b
:1025500000000000001d0000000000002727000010
:1025600000270000c3c30000ff000000c3ff0000fd
:10257000e5000000ffff0000e0000000ffe00000b9
:1025800000e0000000ff0000ffe0000000ff00008e
:10259000e0e0000000ff0000d8000000d8000000cc
:1025a000ffd800001d000000ffff0000ff1d00001d
:1025b00000ff0000ffff000027000000ff270000d1
:1025c00027000000c3c30000c3000000ffe50000b7
:1025d00000e0000000ff0000ffe0000000ff00003e
:1025e000e0000000e0000000ffff0000ffe000004e
:1025f000e0ff0000e0000000ffd8000000d800006d
:1026000000ff00001d1d000000ff0000ffff000094
:102610001d000000ffff0000ff27000000ff00007a
:102620002727000000c30000c3c3000000ff000014
:10263000e5000000e0000000ffff0000e0000000f7
:10264000ffe0000000e0000000ff0000ffff0000ce
:10265000e0e0000000e0000000ff0000d800000003
:10266000d8000000ff1d00001d000000ffff00005b
:10267000ff1d000000ff0000ffff0000270000001a
:10268000ff27000027000000c3c30000c3000000b4
:10269000ffe5000000e0000000ff0000ffe0000098
:1026a00000ff0000e0000000e0000000ffff00006d
:1026b000ffe00000e0000000e5000000ffd800009f
:1026c00000d8000000ff00001d1d000000ff0000fa
:1026d000ffff00001d000000ffff0000ff270000bb
:1026e00000ff00002727000000c30000c3c3000054
:1026f00000ff0000e5000000e0000000ffff000018
:10270000e0e00000e0e0000000ff0000e0e000008a
:10271000e0e00000ffe0000000e5000000ff000036
:10272000d8000000d8000000ff1d0000001d0000c0
:102730001d1d00001d1d000000ff0000ffff000028
:1027400027000000ff270000c3000000c3c30000f3
:10275000c3000000ffe0000000e0000000ff0000f8
:10276000ffe0000000000000e0000000e0ff0000cb
:102770000000000000e00000e0000000e5d80000dc
:10278000d8d8000000d8000000ff00001d1d000088
:10279000ff000000000000001d000000ffff00001f
:1027a000ff27000000ff000027c3000000c3000057
:1027b000c3c30000e5e50000e0000000e000000009
:1027c000ffff0000e0000000ffe0000000e000006c
:1027d00000ff0000ffff0000e0e0000000d8000064
:1027e00000000000d8000000d8000000ff1d00001d
:1027f0001d000000ffff0000ff1d000000ff0000a3
:10280000ffff000027000000ff270000c3000000ba
:10281000c3c30000c300000000e0000000e00000af
:1028200000ff0000ffe0000000ff0000e0000000eb
:10283000e0000000ffff0000ffe00000e5000000f6
:10284000d8000000ffd8000000d8000000ff000002
:102850001d1d000000ff0000ffff00001d00000024
:10286000ffff0000ff27000000ff0000c3c30000bf
:1028700000c30000c3e5000000ff0000e00000000e
:10288000e0000000ffff0000e0000000ffe00000ab
:1028900000e0000000ff0000ffe00000ff0000007b
:1028a000d8d8000000ff0000d80000001d00000084
:1028b000ff1d00001d000000ffff0000ff1d0000c5
:1028c00000ff0000ffff000027000000ffc3000022
:1028d000c3000000c3c30000e5000000ffe00000eb
:1028e00000e0000000ff0000ffe0000000ff00002b
:1028f000e0000000e0000000ffff0000e00000003a
:10290000ffd80000d8000000ffd80000001d000024
:1029100000ff00001d1d000000ff0000ffff000081
:102920001d000000ffff0000ff27000000ff000067
:10293000c3c3000000c30000e5e5000000ff000085
:10294000e0000000e0000000ffff0000e0000000e9
:10295000ffe0000000ff0000e0e00000e0e0000019
:1029600000ff0000d8d8000000ff0000d8000000e1
:102970001d1d00001dff0000001d00001d1d0000aa
:102980001dff000027270000272700002727000041
:10299000c3c3000000c30000ffe50000e500000025
:1029a000ffe0000000ff0000e0e00000e0ff0000aa
:1029b00000ff0000ff000000ffff0000000000001b
:1029c00000000000ffff000000000000ffff00000b
:1029d00000ff00000000000000ff0000ff000000fa
:1029e0000000000000ff00000000000000000000e8
:1029f0000000000000000000ff000000ff000000d9
:102a000000ff0000ff000000ffff000000000000ca
:102a1000ffff0000ffff0000ffff0000ffff0000be
:102a2000ffff0000ffff0000ffff0000ffff0000ae
:102a3000ffff0000ffff0000ffff0000ffff00009e
:102a4000ffff0000ffff0000ffff0000ffff00008e
:102a5000ffff0000ffff0000ffff0000ffff00007e
:102a6000ffff0000ffff0000ffff0000ffff00006e
:102a7000ffff0000ffff0000ffff0000ffff00005e
:102a8000ffff0000ffff0000ffff0000d8d800009c
:102a9000ff1d0000ffff00001d1d00001d1d0000a8
:102aa0001dff00001d1d0000272700002727000034
:102ab000ff270000ffc30000c3c30000ffff0000aa
:102ac000ffff0000ffff0000ffff0000ffff00000e
:102ad000ffff0000ffff0000ffff0000ffff0000fe
:102ae000ffff0000ffff0000ffff0000d8ff000015
:102af00000d800001d000000ffff0000001d0000c6
:102b0000000000001dff0000000000000027000082
:102b100027000000c3c30000ff0000000000000009
:102b2000ffff0000ffff0000ffff0000ffff0000ad
:102b3000ffff0000ffff0000ffff0000ffff00009d
:102b4000ffff0000ffff0000ffff0000ffd80000b4
:102b500000ff00001d1d000000ff0000ffff00003f
:102b60001d000000ff1d000000ff0000ffff00002f
:102b70002727000000c30000c3000000ffff000083
:102b8000ffff0000ffff0000ffff0000ffff00004d
:102b9000ffff0000ffff0000ffff0000ffff00003d
:102ba000ffff0000ffff0000ffff0000ffff00002d
:102bb000d8000000ff1d00001d000000ffff000006
:102bc000ff1d000000ff00001d000000ffff0000cf
:102bd000ff27000027000000c3c3000000ff000023
:102be000ffff0000ffff0000ffff0000ffff0000ed
:102bf000ffff0000ffff0000ffff0000ffff0000dd
:102c0000ffff0000ffff0000ffff0000ffff0000cc
:102c1000ffd8000000ff00001d1d000000ff0000a5
:102c2000ffff00001d000000ff1d000000ff00006e
:102c3000ffff00002727000000c30000c3000000c2
:102c4000ffff0000ffff0000ffff0000ffff00008c
:102c5000ffff0000ffff0000ffff0000ffff00007c
:102c6000ffff0000ffff0000ffff0000ffff00006c
:102c7000ffff0000d8000000ff1d00001d00000045
:102c8000ffff0000ff1d000000ff00002700000004
:102c9000ffff0000ff270000c3000000c3c30000c7
:102ca00000ff0000ffff0000ffff0000ffff00002b
:102cb000ffff0000ffff0000ffff0000ffff00001c
:102cc000ffff0000ffff0000ffff0000ffff00000c
:102cd000ffff0000ffd8000000ff00001d1d0000e6
:102ce00000ff0000ffff00001d000000ffff0000cc
:102cf000272700002727000027c3000000c300008b
:102d000000c30000e5e50000ffff0000ffff00003a
:102d1000ffff0000ffff0000ffff0000ffff0000bb
:102d2000ffff0000ffff0000ffff0000ffff0000ab
:102d3000ffff0000ffff0000d81d00001d1d000068
:102d40001d000000ffff0000ff1d000000ff00004d
:102d500027ff00000000000000270000c300000063
:102d6000c3000000ff000000e5000000ffff0000be
:102d7000ffff0000ffff0000ffff0000ffff00005b
:102d8000ffff0000ffff0000ffff0000ffff00004b
:102d9000ffff0000ffff0000ffd800000000000060
:102da0001d1d000000ff0000ffff00001d000000cf
:102db000ff27000000ff0000ffff0000c3c300006a
:102dc00000c3000000ff0000ffff0000e0ff000064
:102dd000ffff0000ffff0000ffff0000ffff0000fb
:102de000ffff0000ffff0000ffff0000ffff0000eb
:102df000ffff0000ffff0000ffff00001d000000bc
:102e0000ff1d00001d000000ffff0000ff1d00006f
:102e100000ff000027000000ffff0000ffc30000cc
:102e2000c3000000c3000000ffff0000ffe000003f
:102e300000ff0000ffff0000ffff0000ffff000099
:102e4000ffff0000ffff0000ffff0000ffff00008a
:102e5000ffff0000ffff0000ffff0000ff1d00005c
:102e600000ff00001d1d000000ff0000ffff00002c
:102e70001d000000ff27000000ff0000ffff000012
:102e8000c3c3000000c3000000ff0000ffff0000fc
:102e9000e0000000ffff0000ffff0000ffff000058
:102ea000ffff0000ffff0000ffff0000ffff00002a
:102eb000ffff0000ffff0000ffff0000ffff00001a
:102ec0001d000000ff1d00001d000000ffff0000ae
:102ed000ff1d000000ff000027000000ffff0000b2
:102ee000ffc30000c3000000c3000000ffff00009c
:102ef000e0ff000000ff0000ffff0000ffff0000f8
:102f0000ffff0000ffff0000ffff0000ffff0000c9
:102f1000ffff0000ffff0000ffff0000ffff0000b9
:102f2000ff1d000000ff00001d0000001d1d00002f
:102f30001d1d00002727000027ff00002727000095
:102f4000c3c30000c3000000c3e50000e5e00000cb
:102f5000e0e0000000ff0000ffff0000ffff0000b6
:102f6000ffff0000ffff0000ffff0000ffff000069
:102f7000ffff0000ffff0000ffff0000ffff000059
:102f8000ffff0000ff000000ffff000000ff000047
:102f900000000000000000000000000000ff000032
:102fa000000000000000000000ff00000000000022
:102fb0000000000000000000ffff0000ffff000015
:102fc000ffff0000ffff0000ffff0000ffff000009
:102fd000ffff0000ffff0000ffff0000ffff0000f9
:102fe000ffff0000ffff0000ffff0000ffff0000e9
:102ff000ffff0000ffff0000ffff0000ffff0000d9
:10300000ffff0000ffff0000ffff0000ffff0000c8
:10301000ffff0000ffff0000ffff0000ffff0000b8
:10302000ffff0000ffff0000ffff0000ffff0000a8
:10303000ffff0000ffff0000ffff0000ffff000098
:10304000ffff0000ffff0000ffff0000ffff000088
:10305000ffff0000ffff0000ffff0000ffff000078
:10306000ffff0000ffff0000ffff0000ffff000068
:10307000ffff0000ffff0000ffff0000ffff000058
:10308000ffff0000ffff0000ffff0000ffff000048
:10309000ff1d0000100800000000000025250000b2
:1030a000252500002525000029250000000000003e
:1030b000252500002525000005250000050000004d
:1030c00000000000000000000025000025050000b1
:1030d00005000000006f0000737300004f730000d4
:1030e0004f73000073000000007300007373000052
:1030f00073730000737300002500000000290000b6
:1031000073730000737300004f7300007325000099
:103110006f730000736f0000736f00002a7300006c
:1031200000000000737300007373000073730000ed
:1031300073290000000000002a7300007373000070
:103140007373000073730000256f00007373000039
:103150006f4e00006f4f000073000000007300000e
:10316000734f00004a4a0000737300002a000000f9
:10317000004a000073730000734e00007373000078
:10318000732500006f73000073250000004a0000e3
:1031900073730000000000007373000073000000f0
:1031a000257300006f4a0000000000004e7300000d
:1031b000734f0000002500006f730000294f0000ce
:1031c000737300004a0000004f730000730000009a
:1031d0000073000073730000002900007373000087
:1031e0004a000000004e0000737300004e00000013
:1031f000000500004a0000004f730000732a000021
:10320000004f000073730000000000006f730000a7
:103210007300000029730000734a000000000000e2
:103220004f730000732a000000000000000000003f
:10323000006f0000737300002a0000004f7300004d
:1032400073000000006f0000734f000000290000b1
:10325000737300004a000000004f00007373000009
:10326000736f00004f4f00004f2500004f730000a8
:10327000732a0000004f000073730000000000007c
:103280006f7300007300000025730000734a000094
:10329000000000004f730000734f00006f4f0000ec
:1032a0004f6f0000294f0000737300002a000000d8
:1032b0004f73000073000000006f00007373000084
:1032c00000250000737300004e000000004f000056
:1032d00073730000737300006f4e00004f250000f1
:1032e0004f73000073290000004f0000737300004b
:1032f000000000006f7300007300000029730000dd
:10330000734e0000000000004f7300006f2a0000a1
:103310000000000000000000004f00007373000078
:103320002a0000004f73000073000000006f0000cf
:103330007373000000250000737300004e0000004e
:10334000004f0000737300002500000005250000f9
:10335000250000006f730000732a0000044f000076
:10336000737300000000000073730000730000001e
:1033700025730000734e0000000000004e73000033
:1033800073290000006f0000737300002a730000af
:103390007373000073730000737300006f0000000c
:1033a00000730000737300000025000073730000b9
:1033b0004f000000004e00007373000073730000a4
:1033c00073730000732a00004f73000073730000d2
:1033d00073730000734f0000000000006f73000063
:1033e0007300000029730000734f0000000000000c
:1033f0004e7300007373000073730000737300005a
:103400004a4a0000734f00006f6f0000734f0000c6
:103410004a000000004f0000734f0000002500002c
:103420004f4f00004f000000004a00002a2a000011
:10343000737300006f4f000073250000311000000f
:103440000800000000000000000000000000000074
:10345000000000000000000000000000080c000058
:10346000081000001014000004000000001c000000
:103470000c04000000000000080c00003c080000e4
:1034800000000000080400000c0c00000c08000004
:103490000400000000040000101000000c0c0000ec
:1034a0000400000000000000001800005d1c000087
:1034b00000000000000000000000000014140000e4
:1034c000181c00005d3c00005d10000000000000c2
:1034d0001c7e00007e080000005d00007e5d000094
:1034e00008000000145d00005d7e00005d3c0000ef
:1034f0007e5d00000c0000001c7e00005d3c0000b2
:103500003c1c00001c1c0000000000003c5d000092
:103510007e0000000000000000000000001000001d
:10352000181800003c3c00001c5d00001c0000005e
:10353000003c00007e7e0000080800007e7e000047
:103540007e040000001800005d5d00007e5d00004c
:103550005d7e00007e100000001c00007e5d00000b
:103560003c3c00001c1c000018000000007e000015
:103570007e7e00000000000000000000000000004f
:1035800010180000181000000c3c00007e1c000009
:10359000000000001c7e00007e0c0000005d0000aa
:1035a0007e7e0000000000001c7e00007e7e000089
:1035b0001c5d00007e7e0000100000003c7e0000cc
:1035c0005d1c00001c3c00001c1c000000000000f2
:1035d0007e7e00007e000000000000000000000071
:1035e0000018000018180000080000001c5d000012
:1035f0003c000000001c00007e7e00000c0000006b
:103600007e7e00007e000000001c00007e7e000028
:103610003c000000103c00007e140000003c000054
:103620007e5d0000080000001c3c00001c00000043
:10363000007e00007e7e0000000000000000000010
:10364000000000001814000018080000003c0000f2
:103650005d1c0000000000001c7e00007e080000d1
:10366000007e00007e7e0000000000001c7e000046
:103670007e1c0000000400000c1800000800000080
:103680005d7e00007e040000003c00003c1c000049
:10369000000000007e7e00007e00000000000000b0
:1036a00000000000001800001c18000008000000c6
:1036b0003c5d00001c000000001c00007e7e00003d
:1036c0000c0000005d7e00005d000000001c00009a
:1036d0007e7e0000180000000000000000000000d6
:1036e000005d00007e7e00000c0400003c3c0000f9
:1036f00010000000007e00007e7e00000000000040
:103700000000000000000000141c00001c08000065
:10371000001c00005d1c0000000000001c7e00007a
:103720007e5d00003c7e00007e7e00000000000008
:103730003c7e00007e7e00005d1c00001c3c000002
:10374000100000007e7e00007e1c00001c3c00007b
:103750001c000000000000007e7e00007e000000d3
:103760000000000000000000001800001c1c000009
:103770000c0800003c3c000018000000001c000089
:103780007e7e00007e7e00007e7e00005d000000e8
:10379000003c00005d5d00003c5d00001c3c000042
:1037a0005d140000005d00007e5d00005d7e000095
:1037b0005d1c000000000000007e00007e7e000016
:1037c0000000000000000000000000001c1c0000c1
:1037d0001c3c00003c3c00005d14000000000000a8
:1037e000040800001c7e00007e7e00007e080000b1
:1037f000000000003c7e00005d7e00005d5d00007a
:103800001c1c0000100000005d7e00007e3c0000db
:103810005d5d00007e140000000000007e7e000060
:103820007e000000001c00003c1c00000010000096
:103830005d1c00001c3c00003c3c0000140000002b
:1038400000000000001c00007e7e00007e100000d2
:1038500000000000003c00005d5d00001804000056
:103860000404000008000000005d00007e7e0000ef
:10387000100800007e5d00005d000000007e00007a
:103880007e7e0000000000007e7e00007e000000c2
:103890000c5d000018100000145d00001c140000f6
:1038a00000000000000000001c7e00007e3c0000c4
:1038b00000000000000000001c5d00007e10000001
:1038c000000c000010140000040000005d7e0000e9
:1038d0007e100000087e00007e7e000000000000d8
:1038e0007e7e00007e040000047e00007e7e0000dc
:1038f000001000001c1c0000040c00001c1c000038
:103900001c00000000000000001c00007e7e000083
:103910003c00000000000000001c00005d7e000074
:10392000140400003c7e00007e140000005d0000d6
:103930007e7e0000180c00007e7e00005d0400000a
:10394000007e00007e7e00007e7e00007e7e000005
:103950007e000000181c00001c040000081c000071
:103960003c1c000000000000000000001c7e000065
:103970007e3c000000000000000000001c7e0000f3
:103980007e7e00007e5d00007e7e0000180000004c
:103990005d7e00007e180000107e00007e5d00004d
:1039a000080000007e7e00007e7e00007e7e00001b
:1039b0007e7e0000003c00003c1c0000000800006f
:1039c0001c1c00001c00000000000000001800008b
:1039d0007e7e00003c00000000000000001c000093
:1039e0005d7e00005d7e00005d7e00007e180000b0
:1039f000005d00007e7e0000180c00007e7e00004e
:103a00003c080000001c00001c5d00007e7e0000e1
:103a10007e7e00003c000000141c0000140000002a
:103a2000041c0000181c0000000000000000000042
:103a30000c1c00001c18000000000000000000002a
:103a40001c140000147e00005d5d00003c5d000061
:103a5000100000005d7e00005d100000041c0000ee
:103a60003c3c0000081d00001008000000000000a1
:103a70000c100000100c00001010000014100000ca
:103a8000000000000c0c0000100c00000c0c0000ea
:103a90000c0000000000000000080000040c000002
:103aa0000c0c000008040000005d00007e7e000099
:103ab0003d7e00003c7e00005e000000007e0000b5
:103ac0007e7e00005e5e00007e5e00001000000052
:103ad000001400005d5e00007e5e00003d7e000080
:103ae0005e0c00005d7e00007e5d00007e5d0000db
:103af000187e0000000000007e7e00007e5e000058
:103b00007e5e00007e14000000000000185e0000d1
:103b10005e7e00005e5e00007e7e0000105d0000a4
:103b20007e7e00003d1c00005d3c00007e00000029
:103b3000007e00007e3d0000181c00007e5e00003c
:103b400018000000001c00007e7e00007e1c0000ab
:103b50005d7e00007e1000005d7e00005e140000af
:103b6000001c00007e7e0000000000005e7e000061
:103b70007e000000105d00005d1c000000000000e1
:103b80001c7e00007e3c0000001000003d7e000016
:103b9000143d00007e5e00001c0000003c7e000022
:103ba0007e040000005e00007e7e00000014000025
:103bb0005e7e00001c000000001c00007e7e0000f5
:103bc0001c000000040c0000180800003c7e0000ef
:103bd0007e140000003c00007e7e0000000000001b
:103be0005d7e00007e000000145e00007e1c000070
:103bf000000000001c7e00007e1800000000000095
:103c000000000000003d00007e7e00001800000063
:103c10003c7e00007e000000005d00007e3d000054
:103c2000001400007e7e00001c000000003c00002c
:103c30007e7e00007e5d00001c1c00003c10000029
:103c40003d7e00007e180000003c00007e7e0000eb
:103c5000000000005d7e00007e000000145e000099
:103c60005e180000000000003c5d00005e3d0000aa
:103c70005d1c00003c5d0000143d00007e7e0000e5
:103c8000140000003c7e00007e000000005d00008b
:103c90007e5e0000001000007e7e00001c00000020
:103ca000003d00007e5e00007e5e00005d1c0000a6
:103cb0001c1000003c7e00007e140000001c000070
:103cc0007e7e0000000000005d7e00007e0000009f
:103cd000147e00007e1c0000000000003c5e00001e
:103ce0005d1800000404000004080000003c00000f
:103cf0007e7e0000180000003c7e00007e00000078
:103d0000005d00007e7e0000001000007e7e00004e
:103d10001c000000001c00005e7e0000100000007f
:103d20000c100000140400005d7e00007e180000ee
:103d3000083c00007e5e0000000000005d7e000088
:103d40005e000000107e00007e1c000000000000ed
:103d50001c5e00007e140000043d00007e7e00001a
:103d6000145e00007e7e00007e7e00007e7e0000ed
:103d70005d000000005d00007e7e00000410000079
:103d80007e7e00003c000000001c00007e7e0000e3
:103d90007e7e00005e7e00007e1800003c7e0000fb
:103da0007e7e00007e7e00007e3c00000000000061
:103db0005d7e00007e040000147e00007e3c00005a
:103dc000000000001c5d00007e5d00007e5e0000c3
:103dd0007e7e0000181c00005d3d00003d5d00007f
:103de0005e3c00001c000000003d00005d3d000046
:103df000041000003d3d00003c000000001c0000dd
:103e0000141400007e5d00005d3d00005d100000a8
:103e10000d0e000008e3000000e3000000e30000d6
:103e2000e3e30000e3e3000000e30000e3e300005d
:103e3000e3e3000000f2000000e30000e3e3000021
:103e400000f2000000e30000e3e30000e3000000f4
:103e5000f20000000000000000000000f20000007e
:103e6000e3e30000e3e300000000000000000000c6
:103e7000000000000000000000e30000e3e3000099
:103e8000e3000000fcfc00000000000000fc00005b
:103e9000fc000000e3e30000e3e30000000000009a
:103ea00000000000f20000000000000000e300003d
:103eb000e3e30000e3e30000006d00006d0000009c
:103ec0006d6d000000e30000e3e30000e3e30000a9
:103ed000e3e30000000000000000000000e3000039
:103ee000e3e30000e3e30000e3e30000e30000009d
:103ef000ffff0000ff000000e3e30000e3e3000039
:103f0000e3e30000e300000000ff0000ffff00000b
:103f100000000000e300000000000000e3e30000f8
:103f20000000000000ff00000000000000e30000af
:103f300000e3000000e30000e300000000000000d8
:103f40000000000000000000e3e30000e3000000c8
:103f5000e3e300000000000000000000000000009b
:103f6000000000000000000000e30000e3e30000a8
:103f700000000000e300000000e30000e3e30000b5
:103f8000e3e30000e30d00000e080000e300000082
:103f9000e3000000e3e30000e3e30000e3000000cf
:103fa000e3e30000e3e30000e3000000f2000000b0
:103fb000e3e30000e3000000f2000000e3e30000a0
:103fc000e3e3000000f20000000000000000000039
:103fd00000f2000000e30000e3e30000e300000063
:103fe00000000000000000000000000000000000d1
:103ff000e3e30000e3e3000000fc0000fc0000003d
:1040000000000000fcfc000000e30000e3e300000f
:10401000e30000000000000000f2000000000000cb
:1040200000000000e3e30000e3e30000e300000021
:104030006d6d0000006d00006d000000e3e3000006
:10404000e3e30000e3e30000e30000000000000001
:1040500000000000e3e30000e300000000e30000d4
:10406000e3e3000000ff0000ffff000000e30000aa
:10407000e3e30000e3000000e3e3000000000000d1
:10408000ffff0000ff00000000e30000e3e300008a
:1040900000e30000e300000000000000ff0000005b
:1040a00000000000e3e30000e3000000e3e30000a1
:1040b00000000000000000000000000000e300001d
:1040c000e3e3000000e30000e30000000000000064
:1040d00000000000000000000000000000000000e0
:1040e000e3e30000e300000000e300000000000044
:1040f000e3e30000e3e30000e3e300000d0e000053
:1041000008e3000000e3000000e30000e3e3000038
:10411000e3e3000000e30000e3e30000e3e300006a
:1041200000f2000000e30000e3e3000000f2000002
:1041300000e30000e3e30000e3000000f200000001
:104140000000000000000000f2000000e3e30000b7
:10415000e3e3000000000000000000000000000099
:104160000000000000e30000e3e30000e3000000c3
:10417000fcfc00000000000000fc0000fc0000004f
:10418000e3e30000e3e300000000000000000000a3
:10419000f20000000000000000e30000e3e3000084
:1041a000e3e30000006d00006d0000006d6d000095
:1041b00000e30000e3e3000000e30000e3e30000ad
:1041c000000000000000000000e30000e3e3000046
:1041d000e3000000e3e30000e3000000ffff000055
:1041e000ff000000e3e30000e3e3000000e3000061
:1041f000e300000000ff0000ffff000000000000df
:10420000e3e30000e3000000e3e30000000000003f
:1042100000ff00000000000000e30000e3e30000f6
:1042200000e30000e30000000000000000000000c8
:1042300000000000e3e30000e3000000e3e300000f
:10424000000000000000000000000000000000006e
:104250000000000000e30000e3e3000000000000b5
:10426000e300000000e30000e3e30000e3e30000fc
:10427000e30d00000e080000e3000000e300000072
:10428000e3e30000e3e30000e3000000e3e30000f9
:10429000e3e30000e3000000f2000000e3e30000bd
:1042a000e3000000f2000000e3e30000e3e30000ad
:1042b00000f20000000000000000000000f200001a
:1042c00000e30000e3e30000e30000000000000062
:1042d000000000000000000000000000e3e3000018
:1042e000e3e3000000fc0000fc0000000000000010
:1042f000fcfc000000e30000e3e30000e30000003a
:104300000000000000f200000000000000000000bb
:10431000e3e30000e3e30000e30000006d6d000054
:10432000006d00006d000000e3e30000e3e3000027
:10433000e3e30000e30000000000000000000000d4
:10434000e3e30000e3e3000000000000e3e300001b
:1043500000ff0000ffff000000e30000e3e30000b7
:10436000e3000000e3e3000000000000ffff0000a6
:10437000ff00000000e30000e3e3000000e30000b2
:10438000e300000000000000ff000000000000004b
:10439000e3e30000e3000000e3e3000000000000ae
:1043a000000000000000000000e30000e3e3000064
:1043b00000e30000e3000000000000000000000037
:1043c000000000000000000000000000e3e3000027
:1043d000e300000000e3000000000000e3e3000051
:1043e000e3e30000e3e300004f4f000008e30000b8
:1043f00000e00000e0e00000e1e10000e1e1000099
:10440000e2e20000e2e20000e3e30000e3e3000098
:10441000e3c30000c3c30000a3a300008383000024
:104420008383000063630000634300004343000094
:104430004343000043230000232300002323000004
:104440002323000023230000232300002323000054
:104450004343000043430000434300006363000004
:10446000638300008383000083a30000a3c30000d4
:10447000c3c30000e3e30000e3e30000e3e2000065
:10448000e2e20000e2e10000e1e10000e1e0000022
:10449000e0e00000e1e10000e1e10000e2e2000014
:1044a000e2e30000e3e30000e3e30000c3c3000035
:1044b000c3a30000a38300008383000063630000a4
:1044c0006343000043430000432300002323000014
:1044d0002323000023230000232300000303000004
:1044e0000303000003230000232300002323000014
:1044f0002323000023230000434300004343000024
:10450000636300006383000083830000a3a30000b3
:10451000c3c30000c3e30000e3e30000e3e20000e4
:10452000e2e20000e2e10000e1e10000e1e0000081
:10453000e1e10000e1e10000e2e20000e2e300006e
:10454000e3e30000e3e30000c3c30000c3a30000f3
:10455000a383000083630000636300004343000003
:104560004323000023230000232300000303000053
:104570000303000003030000030300000303000023
:104580000303000003030000030300000303000013
:1045900003230000232300002323000043430000e3
:1045a000436300006363000083830000a3a3000053
:1045b000c3c30000c3e30000e3e30000e3e3000043
:1045c000e2e20000e2e10000e1e10000e1e10000e0
:1045d000e1e10000e2e20000e2e30000e3e30000ca
:1045e000e3c30000c3c30000a3a300008383000053
:1045f0008363000063430000434300002323000063
:104600002323000003030000030300000303000052
:104610000303000003030000030300000303000082
:104620000303000003030000030300000303000072
:1046300003030000032300002323000023430000a2
:1046400043430000636300008383000083a30000f2
:10465000a3c30000c3c30000e3e30000e3e30000e2
:10466000e2e20000e2e10000e1e10000e1e100003f
:10467000e2e20000e2e30000e3e30000e3c3000045
:10468000c3c30000a3a30000838300006363000092
:1046900043430000432300002323000003030000e2
:1046a00003030000030300000303000007070000ea
:1046b00007070000070700000707000007070000c2
:1046c00007070000070700000703000003030000be
:1046d0000303000003030000032300002323000062
:1046e00043430000436300006383000083a3000092
:1046f000a3c30000c3c30000e3e30000e3e3000042
:10470000e2e20000e2e10000e1e10000e2e200009c
:10471000e2e30000e3e30000e3c30000c3c30000e2
:10472000a383000083830000634300004343000031
:104730002323000023030000030300000303000001
:104740000307000007070000070700000b0b00002d
:104750000b0b00000b0b00000b0b00000b0b000001
:104760000b0b00000b070000070700000707000005
:1047700003030000030300000303000023230000e1
:104780002343000043430000638300008383000051
:10479000a3c30000c3c30000e3e30000e3e30000a1
:1047a000e2e20000e2e10000e2e20000e2e30000f9
:1047b000e3e30000e3c30000c3a30000a383000001
:1047c00083630000634300004323000023230000b1
:1047d00003030000030300000307000007070000b5
:1047e000070b00000b0b00000b0b00000b0f000071
:1047f0000f0f00000f0f00000f0f00000f0f000041
:104800000b0b00000b0b00000b0b00000707000058
:104810000707000003030000030300000323000058
:1048200023230000434300006363000083830000f0
:10483000a3a30000c3c30000e3e30000e3e3000020
:10484000e2e20000e2e20000e2e30000e3e3000055
:10485000e3c30000c3a30000a38300008363000040
:1048600063430000432300002323000003030000f0
:104870000303000007070000070b00000b0b0000fc
:104880000b0f00000f0f00000f13000013130000a8
:104890001313000013130000131300001313000080
:1048a0000f0f00000f0f00000b0b00000b0b0000a0
:1048b00007070000070300000303000003230000b4
:1048c0002323000043430000636300008383000050
:1048d000a3a30000c3c30000e3e30000e3e3000080
:1048e000e2e20000e2e30000e3e30000e3c30000d3
:1048f000c3a30000a38300008363000043430000c0
:10490000432300002303000003030000030700000b
:10491000070700000b0b00000b0f00000f0f00003b
:1049200013130000131300001317000017170000e3
:1049300017170000171700001717000013130000c7
:1049400013130000130f00000f0f00000b0b0000eb
:104950000b0700000707000003030000030300002b
:1049600023230000434300004363000083830000cf
:10497000a3a30000c3c30000e3e30000e3e30000df
:10498000e2e20000e3e30000e3c30000c3a3000091
:10499000a38300008363000043430000232300003f
:1049a000230300000303000003070000070b0000bf
:1049b0000b0b00000f0f0000131300001317000073
:1049c0001717000017170000171b00001b1b000023
:1049d0001b1b00001b1b000017170000171700000f
:1049e0001717000013130000130f00000f0b000037
:1049f0000b0b000007070000030300000303000087
:104a0000232300002343000043630000838300004e
:104a1000a3a30000c3c30000e3e30000e3e200003f
:104a2000e3e30000e3c30000c3a30000a38300008e
:104a300083630000434300002323000003030000be
:104a400003030000070700000b0b00000b0f000022
:104a50000f1300001317000017170000171b0000aa
:104a60001b1b00001b1b00001b1b00001b1b00006e
:104a70001b1b00001b1b00001b1b00001b1b00005e
:104a80001717000017170000131300000f0f000086
:104a90000b0b00000b0700000703000003030000de
:104aa00003230000234300004363000083830000ce
:104ab000a3a30000c3c30000e3e30000e3e300009e
:104ac000e3c30000c3c30000a383000083630000ae
:104ad00043430000232300000303000003030000fe
:104ae000070700000b0b00000f0f0000131300005e
:104af00017170000171b00001b1b00001b1f0000e6
:104b00001f1f00001f1f00001f1f00001f1f0000ad
:104b10001f1f00001f1f00001f1f00001b1b0000a5
:104b20001b1b00001717000017130000130f0000d5
:104b30000f0b00000b070000070300000303000039
:104b4000032300002343000043630000838300002d
:104b5000a3c30000c3c30000e3e30000e3e30000dd
:104b6000c3c30000a383000083630000434300002d
:104b700023230000030300000303000007070000d5
:104b80000b0b00000f130000131700001717000095
:104b90001b1b00001b1f00001f1f00001f1f000029
:104ba0001f1f00001f1f00001f1f00001f1f00000d
:104bb0001f1f00001f1f00001f1f00001f1f0000fd
:104bc0001b1b00001b170000171700001313000029
:104bd0000f0b00000b070000070300000303000099
:104be000032300002343000043630000838300008d
:104bf000a3c30000c3e30000e3e30000c3c300005d
:104c0000a3830000836300004343000023230000cc
:104c10000303000003070000070b00000b0f000058
:104c20000f13000013170000171b00001b1b0000d0
:104c30001f1f00001f1f00001f1f00001f1f00007c
:104c40001f1f00001f1f00001f1f00001f1f00006c
:104c50001f1f00001f1f00001f1f00001f1f00005c
:104c60001f1b00001b1b0000171700001313000080
:104c70000f0f00000b0b00000707000003030000ec
:104c800003230000234300004363000083830000ec
:104c9000a3c30000c3e30000c3c30000a3a300003c
:104ca000836300006343000023230000030300002c
:104cb00003070000070b00000b0f00000f1300009c
:104cc000171700001b1b00001b1f00001f1f000008
:104cd0001f1f00001f1f00001f1e00001e1e0000df
:104ce0001e1e00001e1e00001e1e00001e1e0000d4
:104cf0001e1e00001f1f00001f1f00001f1f0000be
:104d00001f1f00001b1b00001b17000017130000d3
:104d10000f0f00000b0b000007070000030300004b
:104d200003230000234300006363000083a300000b
:104d3000a3c30000e3c30000c3a3000083830000fb
:104d40006343000043230000030300000307000047
:104d5000070b00000b0f00001313000017170000d3
:104d60001b1b00001f1f00001f1f00001f1f000053
:104d70001f1e00001e1e00001e1e00001e1e000042
:104d80001e1e00001e1e00001e1e00001e1e000033
:104d90001e1e00001e1e00001f1f00001f1f00001f
:104da0001f1f00001f1b00001b170000171300002f
:104db000130f00000b0b00000707000003030000a7
:104dc00003230000434300006383000083a300002b
:104dd000c3c30000c3a3000083830000634300003b
:104de000432300002303000003030000070b00001f
:104df0000b0f000013130000171700001b1b00000f
:104e00001f1f00001f1f00001f1f00001e1e0000ac
:104e10001e1e00001e1e00001e1e00001e1e0000a2
:104e20001e1e00001e1e00001e1e00001e1e000092
:104e30001e1e00001e1e00001e1f00001f1f00007f
:104e40001f1f00001f1b00001b170000171300008e
:104e5000130f00000b0b000007030000030300000a
:104e600023230000434300006383000083a300006a
:104e7000c3a30000a383000063430000432300009a
:104e80002303000003030000070b00000b0f0000ca
:104e900013130000171b00001b1f00001f1f000042
:104ea0001f1f00001f1e00001e1e00001e1e00000f
:104eb0001e1e00001e1d00001d1d00001d1d000007
:104ec0001d1d00001d1d00001d1d00001e1e0000f8
:104ed0001e1e00001e1e00001e1e00001f1f0000e0
:104ee0001f1f00001f1f00001b1b000017130000e6
:104ef000130f00000b0b000007030000030300006a
:104f0000232300004343000063830000a3c3000089
:104f1000a3830000836300004323000023030000f9
:104f200003030000070700000b0f0000131300002d
:104f3000171b00001b1f00001f1f00001f1f000089
:104f40001e1e00001e1e00001e1e00001e1d000072
:104f50001d1d00001d1d00001d1d00001d1d000069
:104f60001d1d00001d1d00001d1d00001d1d000059
:104f70001e1e00001e1e00001e1e00001e1f000040
:104f80001f1f00001f1f00001b1b00001713000045
:104f9000130f00000b0700000703000003030000cd
:104fa000232300004363000083830000a3a30000c9
:104fb0008363000043430000232300000303000039
:104fc000070700000b0f00000f130000171b000065
:104fd0001b1f00001f1f00001f1f00001e1e0000df
:104fe0001e1e00001e1d00001d1d00001d1d0000d6
:104ff0001d1d00001d1d00001d1d00001d1d0000c9
:105000001d1d00001d1d00001d1d00001d1d0000b8
:105010001d1d00001e1e00001e1e00001e1f0000a1
:105020001f1f00001f1f00001b1b000017130000a4
:105030000f0f00000b070000070300000323000010
:10504000234300004363000083a300008363000048
:105050006343000023230000030300000307000054
:105060000b0b00000f130000171700001b1f0000a0
:105070001f1f00001f1f00001e1e00001e1e00003c
:105080001e1d00001d1d00001d1d00001d1c000038
:105090001c1c00001c1c00001c1c00001c1c000030
:1050a0001c1c00001c1c00001d1d00001d1d00001c
:1050b0001d1d00001e1e00001e1e00001e1f000001
:1050c0001f1f00001f1f00001b1700001713000008
:1050d0000f0b00000b070000030300000323000078
:1050e00023430000636300008383000063430000e8
:1050f0004323000003030000030700000b0b000024
:105100000f130000171700001b1f00001f1f0000d7
:105110001f1f00001e1e00001e1e00001d1d00009f
:105120001d1d00001d1d00001c1c00001c1c00009b
:105130001c1c00001c1c00001c1c00001c1c00008f
:105140001c1c00001c1c00001c1d00001d1d00007c
:105150001d1d00001d1e00001e1e00001e1f000061
:105160001f1f00001f1f00001b1700001713000067
:105170000f0b00000b0700000303000003230000d7
:105180004343000063830000636300004323000087
:105190002303000003070000070b00000f130000ab
:1051a000131700001b1b00001f1f00001f1f000023
:1051b0001e1e00001e1e00001d1d00001d1d000003
:1051c0001d1c00001c1c00001c1c00001c1c0000fe
:1051d0001c1c00001c1c00001c1c00001c1c0000ef
:1051e0001c1c00001c1c00001c1c00001d1d0000dd
:1051f0001d1d00001d1e00001e1e00001e1f0000c1
:105200001f1f00001f1b00001b17000013130000ce
:105210000f0b00000707000003030000232300001a
:105220004363000083630000434300002303000046
:1052300003030000070b00000b0f00001317000012
:105240001b1b00001f1f00001f1f00001e1e000070
:105250001e1e00001d1d00001d1d00001c1c000066
:105260001c1c00001c1c00001c1c00003c3c00001e
:105270003c3c00003c3c00003c3c00003c1c00006e
:105280001c1c00001c1c00001c1c00001c1d00003d
:105290001d1d00001d1e00001e1e00001e1f000020
:1052a0001f1f00001f1b00001b170000130f000032
:1052b0000b0b000007030000030300002343000062
:1052c0004383000063430000232300000303000026
:1052d000070700000b0f000013170000171b00004a
:1052e0001f1f00001f1f00001e1e00001e1e0000ca
:1052f0001d1d00001d1d00001c1c00001c1c0000ca
:105300001c1c00003c3c00003c3c00003c5c0000dd
:105310005c5c00005c5c00003c3c00003c3c00002d
:105320003c1c00001c1c00001c1c00001c1d00007c
:105330001d1d00001d1e00001e1e00001e1f00007f
:105340001f1f00001f1b000017170000130f000095
:105350000b070000070300000323000023430000a5
:105360006343000043230000030300000307000021
:105370000b0b00000f130000171b00001b1f000089
:105380001f1f00001e1e00001e1e00001d1d00002d
:105390001d1d00001c1c00001c1c00001c3c00000b
:1053a0003c3c00005c5c00005c5c00005c5c00005d
:1053b0005c5c00005c5c00005c5c00005c3c00002d
:1053c0003c3c00001c1c00001c1c00001c1d0000bc
:1053d0001d1d00001d1e00001e1e00001e1f0000df
:1053e0001f1f00001b1b0000171300000f0b000005
:1053f0000b070000030300000323000043630000c9
:10540000432300002303000003070000070b0000f4
:105410000f130000171700001b1f00001f1f0000c4
:105420001f1e00001e1e00001d1d00001d1d00008f
:105430001c1c00001c1c00001c3c00003c5c00000c
:105440005c5c00007c7c00007c7c00007c7c0000bc
:105450007c7c00007c7c00007c5c00005c5c0000cc
:105460003c3c00001c1c00001c1c00001c1d00001b
:105470001d1d00001d1e00001e1e00001f1f00003d
:105480001f1f00001b170000171300000f0b000068
:10549000070700000303000023230000634300000c
:1054a0002323000003030000070b00000b0f000084
:1054b000131700001b1b00001f1f00001f1e000011
:1054c0001e1e00001e1d00001d1d00001c1c0000f3
:1054d0001c1c00001c3c00003c5c00005c7c0000cc
:1054e0007c7c00009c9c00009c9c00009c9c00001c
:1054f0009c9c00009c7c00007c7c00005c5c0000ac
:105500003c3c00001c1c00001c1c00001c1d00007a
:105510001d1d00001e1e00001e1e00001f1f00009b
:105520001f1b00001b170000130f00000b0b0000d7
:10553000070300000323000023430000432300006f
:1055400003030000030700000b0f00001317000007
:10555000171b00001f1f00001f1f00001e1e000061
:105560001e1d00001d1d00001c1c00001c1c000056
:105570001c3c00003c5c00005c7c00007c9c00004b
:105580009cbc0000bcbc0000bcbc0000bcbc00005b
:10559000bcbc00009c9c00007c7c00005c5c0000ab
:1055a0003c3c00001c1c00001c1c00001c1d0000da
:1055b0001d1d00001e1e00001e1f00001f1f0000fa
:1055c0001f1b000017170000130f00000b0700003f
:1055d0000303000003230000432300002303000013
:1055e00003070000070b00000f130000171b00004b
:1055f0001b1f00001f1f00001e1e00001e1d0000bc
:105600001d1d00001d1c00001c1c00001c3c000097
:105610003c5c00007c7c00009c9c0000bcbc00004a
:10562000bcdc0000dcdc0000dcdc0000dcdc0000ba
:10563000bcbc0000bc9c00009c7c00007c5c0000aa
:105640003c3c00001c1c00001c1c00001d1d000038
:105650001d1d00001e1e00001e1f00001f1f000059
:105660001b1b0000171300000f0b000007070000b2
:105670000303000023430000232300000303000072
:10568000070b00000b0f0000131700001b1f00008a
:105690001f1f00001f1e00001e1e00001d1d000019
:1056a0001d1c00001c1c00001c3c00003c5c000099
:1056b0007c7c00009cbc0000bcbc0000dcdc00006a
:1056c000dcdc0000fcfc0000fcdc0000dcdc00009a
:1056d000dcbc0000bcbc00009c7c00007c5c0000ca
:1056e0003c3c00001c1c00001c1c00001d1d000098
:1056f0001d1e00001e1e00001f1f00001f1f0000b7
:105700001b170000130f00000b0b00000703000025
:1057100003230000432300000303000003070000ed
:105720000b0f000013170000171b00001f1f0000c5
:105730001f1e00001e1e00001e1d00001d1d00007b
:105740001c1c00001c3c00003c5c00005c7c000059
:105750009cbc0000bcdc0000dcdc0000fcfc0000a9
:10576000fcfc0000fcfc0000fcfc0000fcdc000079
:10577000dcdc0000bcbc00009c7c00005c5c000029
:105780003c3c00001c1c00001c1d00001d1d0000f6
:105790001e1e00001e1e00001f1f00001f1b000019
:1057a00017170000130f00000b0700000303000091
:1057b000034300002303000003030000070b000065
:1057c0000f130000171b00001b1f00001f1f00000d
:1057d0001e1e00001e1d00001d1d00001c1c0000e0
:1057e0001c1c00003c5c00005c7c00009cbc0000b9
:1057f000bcdc0000dcfc0000fcfc0000fcfc000049
:10580000f8f80000f8fc0000fcfc0000fcfc0000c4
:10581000dcdc0000bcbc00009c7c00005c5c000088
:105820003c1c00001c1c00001c1d00001d1d000075
:105830001e1e00001e1f00001f1f00001b1b00007b
:10584000171300000f0b0000070300000303000004
:105850004323000003030000070700000b0f0000b4
:10586000131700001b1f00001f1f00001f1e000059
:105870001e1e00001d1d00001d1c00001c1c000041
:105880003c3c00005c7c00007c9c0000bcdc000018
:10589000dcfc0000fcfc0000f8f80000f8f8000058
:1058a000f8f80000f8f80000f8fc0000fcfc00002c
:1058b000dcdc0000bc9c00007c7c00005c3c000048
:1058c0003c1c00001c1c00001d1d00001d1e0000d3
:1058d0001e1e00001f1f00001f1f00001b170000de
:1058e000130f00000b070000070300000323000054
:1058f00023030000030700000b0b00000f13000040
:10590000171b00001f1f00001f1e00001e1e0000ae
:105910001e1d00001d1c00001c1c00001c3c000083
:105920005c5c00007c9c0000bcbc0000dcfc000057
:10593000fcfc0000f8f80000f8f40000f4f40000ab
:10594000f4f40000f8f80000f8fc0000fcfc000093
:10595000dcbc0000bc9c00007c5c00005c3c0000e7
:105960001c1c00001c1c00001d1d00001e1e000051
:105970001e1e00001f1f00001f1b00001713000049
:105980000f0b00000b07000003030000232300009f
:1059900003030000070b00000b0f000013170000ab
:1059a0001b1f00001f1f00001e1e00001e1d000008
:1059b0001d1d00001c1c00001c1c00003c5c0000a5
:1059c0007c7c00009cbc0000dcdc0000fcfc0000d7
:1059d000f8f80000f4f40000f0f00000f0f000002f
:1059e000f0f40000f4f80000f8fc0000fcdc00001b
:1059f000dcbc00009c7c00007c5c00003c1c0000c7
:105a00001c1c00001c1d00001d1d00001e1e0000af
:105a10001e1f00001f1f00001b170000130f0000b7
:105a20000b0b00000703000003230000230300000a
:105a3000030700000b0f000013170000171b0000e6
:105a40001f1f00001f1e00001e1e00001d1d000065
:105a50001d1c00001c1c00003c3c00005c7c000085
:105a60009cbc0000bcdc0000fcfc0000f8f800005e
:105a7000f4f40000f0ec0000ecec0000ecec0000b2
:105a8000f0f40000f4f80000f8fc0000fcdc00007a
:105a9000bcbc00009c7c00005c3c00003c1c000086
:105aa0001c1c00001d1d00001d1e00001e1e00000d
:105ab0001f1f00001f1b000017170000130f00001e
:105ac0000b07000003030000232300000303000072
:105ad000070b00000f130000171b00001b1f000026
:105ae0001f1f00001e1e00001e1d00001d1d0000c7
:105af0001c1c00001c3c00003c5c00007c9c000066
:105b0000bcdc0000dcfc0000fcf80000f8f4000045
:105b1000f0ec0000ece80000e8e80000ecec00002d
:105b2000f0f40000f8f80000fcfc0000dcdc0000f1
:105b3000bc9c00007c5c00003c3c00001c1c000085
:105b40001c1d00001d1d00001e1e00001e1f000069
:105b50001f1f00001b1b0000171300000f0b00008d
:105b600007030000032300000303000003070000f5
:105b70000b0f0000131700001b1b00001f1f00006d
:105b80001f1e00001e1e00001d1d00001d1c000029
:105b90001c1c00003c5c00005c7c00009cbc000005
:105ba000dcdc0000fcfc0000f8f40000f0ec00007d
:105bb000ece80000e4e40000e4e80000ecec0000a5
:105bc000f0f40000f8fc0000fcdc0000dcbc00008d
:105bd0009c7c00005c5c00003c1c00001c1c000065
:105be0001d1d00001d1e00001e1e00001f1f0000c6
:105bf0001f1b00001b170000130f00000b07000005
:105c0000030300002303000003030000070b000050
:105c10000f130000171b00001b1f00001f1f0000b8
:105c20001e1e00001e1d00001d1d00001c1c00008b
:105c30001c3c00005c5c00007c9c0000bcdc0000a4
:105c4000fcfc0000f8f80000f4f00000ece80000b4
:105c5000e4e40000e4e40000e4e80000ecf000000c
:105c6000f4f80000f8fc0000fcdc0000bc9c000024
:105c70007c5c00005c3c00001c1c00001c1d000043
:105c80001d1d00001e1e00001e1f00001f1f000023
:105c90001b1b0000171300000f0b00000703000080
:105ca0000323000003030000030700000b0f0000a4
:105cb000131700001b1b00001f1f00001f1e000009
:105cc0001e1e00001d1d00001d1c00001c1c0000ed
:105cd0003c5c00005c7c00009cbc0000dcfc000024
:105ce000fcf80000f8f40000f0ec0000e8e400002c
:105cf000e4e00000e4e40000e8ec0000f0f4000060
:105d0000f8f80000fcfc0000dcbc00009c7c0000fb
:105d10005c5c00003c1c00001c1c00001d1d000001
:105d20001d1e00001e1e00001f1f00001f1b000084
:105d30001b170000130f00000b07000003030000f7
:105d40002303000003030000070b00000f130000f3
:105d5000171b00001b1f00001f1f00001e1e00005d
:105d60001e1d00001d1d00001c1c00001c3c00002e
:105d70005c5c00007c9c0000bcdc0000fcfc0000c3
:105d8000f8f80000f4f00000ece80000e4e40000a3
:105d9000e4e40000e4e80000ecf00000f4f80000a7
:105da000f8fc0000fcdc0000bc9c00007c5c0000f7
:105db0005c3c00001c1c00001c1d00001d1d0000a0
:105dc0001e1e00001e1f00001f1f00001b1b0000e6
:105dd000171300000f0b000007030000032300004f
:105de00003030000030700000b0f0000131700005f
:105df0001b1b00001f1f00001f1e00001e1e0000b6
:105e00001d1d00001d1c00001c1c00003c5c00004f
:105e10005c7c00009cbc0000dcdc0000fcfc0000a2
:105e2000f8f40000f0ec0000ece80000e4e400000e
:105e3000e4e80000ecec0000f0f40000f8fc0000e6
:105e4000fcdc0000dcbc00009c7c00005c5c000012
:105e50003c1c00001c1c00001d1d00001d1e00003d
:105e60001e1e00001f1f00001f1b00001b1700004c
:105e7000130f00000b0700000303000023230000a2
:105e800003030000070b00000f130000171b0000a6
:105e90001b1f00001f1f00001e1e00001e1d000013
:105ea0001d1d00001c1c00001c3c00003c5c000090
:105eb0007c9c0000bcdc0000dcfc0000fcf8000066
:105ec000f8f40000f0ec0000ece80000e8e8000066
:105ed000ecec0000f0f40000f8f80000fcfc00001e
:105ee000dcdc0000bc9c00007c5c00003c3c000052
:105ef0001c1c00001c1d00001d1d00001e1e0000bb
:105f00001e1f00001f1f00001b1b000017130000b6
:105f10000f0b000007030000032300002303000011
:105f2000030700000b0f000013170000171b0000f1
:105f30001f1f00001f1e00001e1e00001d1d000070
:105f40001d1c00001c1c00003c3c00005c7c000090
:105f50009cbc0000bcdc0000fcfc0000f8f8000069
:105f6000f4f40000f0ec0000ecec0000ecec0000bd
:105f7000f0f40000f4f80000f8fc0000fcdc000085
:105f8000bcbc00009c7c00005c3c00003c1c000091
:105f90001c1c00001d1d00001d1e00001e1e000018
:105fa0001f1f00001f1b000017170000130f000029
:105fb0000b0700000303000023230000030300007d
:105fc000070b00000b0f0000131700001b1f000041
:105fd0001f1f00001e1e00001e1d00001d1d0000d2
:105fe0001c1c00001c1c00003c5c00007c7c0000b1
:105ff0009cbc0000dcdc0000fcfc0000f8f80000a9
:10600000f4f40000f0f00000f0f00000f0f4000004
:10601000f4f80000f8fc0000fcdc0000dcbc000030
:106020009c7c00007c5c00003c1c00001c1c0000f0
:106030001c1d00001d1d00001e1e00001e1f000074
:106040001f1f00001b170000130f00000b0b0000a8
:1060500007030000032300002303000003070000e0
:106060000b0b00000f130000171b00001f1f000088
:106070001f1e00001e1e00001e1d00001d1c000033
:106080001c1c00001c3c00005c5c00007c9c0000b0
:10609000bcbc0000dcfc0000fcfc0000f8f80000c8
:1060a000f8f40000f4f40000f4f40000f8f8000044
:1060b000f8fc0000fcfc0000dcbc0000bc9c000004
:1060c0007c5c00005c3c00001c1c00001c1c0000f0
:1060d0001d1d00001e1e00001e1e00001f1f0000d0
:1060e0001f1b0000171300000f0b00000b07000020
:1060f0000303000043230000030300000707000020
:106100000b0f0000131700001b1f00001f1f0000d3
:106110001f1e00001e1e00001d1d00001d1c000093
:106120001c1c00003c3c00005c7c00007c9c0000cf
:10613000bcdc0000dcfc0000fcfc0000f8f8000007
:10614000f8f80000f8f80000f8f80000f8fc00008b
:10615000fcfc0000dcdc0000bc9c00007c7c00003f
:106160005c3c00003c1c00001c1c00001d1d0000cd
:106170001d1e00001e1e00001f1f00001f1f00002c
:106180001b170000130f00000b070000070300009f
:10619000034300002303000003030000070b00007b
:1061a0000f130000171b00001b1f00001f1f000023
:1061b0001e1e00001e1d00001d1d00001c1c0000f6
:1061c0001c1c00003c5c00005c7c00009cbc0000cf
:1061d000bcdc0000dcfc0000fcfc0000fcfc00005f
:1061e000f8f80000f8fc0000fcfc0000fcfc0000db
:1061f000dcdc0000bcbc00009c7c00005c5c00009f
:106200003c1c00001c1c00001c1d00001d1d00008b
:106210001e1e00001e1f00001f1f00001b1b000091
:10622000171300000f0b000007030000030300001a
:106230004323000003030000030700000b0f0000ce
:1062400013170000171b00001f1f00001f1e000077
:106250001e1e00001e1d00001d1d00001c1c000055
:106260001c3c00003c5c00005c7c00009cbc00000e
:10627000bcdc0000dcdc0000fcfc0000fcfc0000de
:10628000fcfc0000fcfc0000fcdc0000dcdc00008e
:10629000bcbc00009c7c00005c5c00003c3c00003e
:1062a0001c1c00001c1d00001d1d00001e1e000007
:1062b0001e1e00001f1f00001f1b000017170000fc
:1062c000130f00000b07000003030000034300004e
:1062d0002323000003030000070b00000b0f000046
:1062e000131700001b1f00001f1f00001f1e0000cf
:1062f0001e1e00001d1d00001d1c00001c1c0000b7
:106300001c3c00003c5c00007c7c00009cbc00004d
:10631000bcbc0000dcdc0000dcdc0000fcfc00009d
:10632000fcdc0000dcdc0000dcbc0000bcbc0000cd
:106330009c7c00007c5c00003c3c00001c1c0000bd
:106340001c1c00001d1d00001d1e00001e1e000064
:106350001f1f00001f1f00001b170000130f00006d
:106360000b0b000007030000032300004323000081
:106370002303000003070000070b00000f130000b9
:10638000171b00001b1f00001f1f00001e1e000027
:106390001e1d00001d1d00001d1c00001c1c000017
:1063a0001c3c00003c5c00007c7c00009c9c0000cd
:1063b000bcbc0000bcdc0000dcdc0000dcdc00005d
:1063c000dcdc0000bcbc0000bc9c00009c7c00002d
:1063d0007c5c00003c3c00001c1c00001c1c0000fd
:1063e0001d1d00001d1d00001e1e00001e1f0000c0
:1063f0001f1f00001b1b0000171300000f0b0000e5
:1064000007070000030300002343000043230000ac
:1064100003030000030700000b0f00001317000028
:10642000171b00001f1f00001f1f00001e1e000082
:106430001e1d00001d1d00001c1c00001c1c000077
:106440001c3c00003c5c00005c7c00007c9c00006c
:106450009cbc0000bcbc0000bcbc0000bcbc00007c
:10646000bcbc00009c9c00007c7c00005c5c0000cc
:106470003c3c00001c1c00001c1c00001c1d0000fb
:106480001d1d00001e1e00001e1f00001f1f00001b
:106490001f1b000017170000130f00000b07000060
:1064a00003030000032300006343000023230000d4
:1064b00003030000070b00000b0f00001317000080
:1064c0001b1b00001f1f00001f1e00001e1e0000df
:1064d0001e1d00001d1d00001c1c00001c1c0000d7
:1064e0001c3c00003c5c00005c7c00007c7c0000ec
:1064f0009c9c00009c9c00009c9c00009c9c0000bc
:106500009c7c00007c7c00005c5c00003c3c00004b
:106510001c1c00001c1c00001c1d00001d1d000098
:106520001e1e00001e1e00001f1f00001f1b00007b
:106530001b170000130f00000b0b000007030000e7
:106540000323000023630000432300002303000013
:1065500003070000070b00000f13000017170000cf
:106560001b1f00001f1f00001f1e00001e1e00003a
:106570001d1d00001d1d00001c1c00001c1c000037
:106580001c3c00003c5c00005c5c00007c7c00006b
:106590007c7c00007c7c00007c7c00007c7c00001b
:1065a0007c5c00005c5c00003c3c00001c1c0000ab
:1065b0001c1c00001c1d00001d1d00001d1e0000f5
:1065c0001e1e00001f1f00001f1f00001b170000e1
:1065d000171300000f0b0000070700000303000063
:1065e0002323000063430000432300000303000053
:1065f000030700000b0b00000f130000171b000027
:106600001b1f00001f1f00001e1e00001e1e00009a
:106610001d1d00001d1d00001c1c00001c1c000096
:106620001c3c00003c3c00005c5c00005c5c00002a
:106630005c5c00005c5c00005c5c00005c5c00007a
:106640005c3c00003c3c00001c1c00001c1c0000ca
:106650001c1d00001d1d00001d1e00001e1e000050
:106660001e1f00001f1f00001b1b0000171300004f
:106670000f0b00000b0700000303000003230000c2
:106680004383000063430000232300000303000052
:10669000070700000b0f000013170000171b000076
:1066a0001f1f00001f1f00001e1e00001e1e0000f6
:1066b0001d1d00001d1d00001c1c00001c1c0000f6
:1066c0001c1c00003c3c00003c3c00003c5c00000a
:1066d0005c5c00005c5c00003c3c00003c3c00005a
:1066e0003c1c00001c1c00001c1c00001c1d0000a9
:1066f0001d1d00001d1e00001e1e00001e1f0000ac
:106700001f1f00001f1b000017170000130f0000c1
:106710000b070000070300000323000023430000d1
:1067200083630000434300002303000003030000d1
:10673000070b00000b0f0000131700001b1b0000cd
:106740001f1f00001f1f00001e1e00001e1e000055
:106750001d1d00001d1d00001c1c00001c1c000055
:106760001c1c00001c1c00003c3c00003c3c0000c9
:106770003c3c00003c3c00003c1c00001c1c000099
:106780001c1c00001c1c00001c1d00001d1d000026
:106790001d1e00001e1e00001e1f00001f1f000007
:1067a0001f1b00001b170000130f00000b0b000045
:1067b000070300000303000023430000438300009d
:1067c000636300004323000023030000030700006d
:1067d000070b00000f130000131700001b1b000025
:1067e0001f1f00001f1f00001e1e00001e1e0000b5
:1067f0001d1d00001d1d00001d1c00001c1c0000b4
:106800001c1c00001c1c00001c1c00001c1c0000a8
:106810001c1c00001c1c00001c1c00001c1c000098
:106820001c1c00001d1d00001d1d00001d1e000081
:106830001e1e00001e1f00001f1f00001f1b000067
:106840001b170000131300000f0b000007070000c8
:10685000030300002323000043630000a383000020
:10686000634300004323000003030000030700000c
:106870000b0b00000f130000171700001b1f000078
:106880001f1f00001f1f00001e1e00001e1e000014
:106890001d1d00001d1d00001d1d00001c1c000012
:1068a0001c1c00001c1c00001c1c00001c1c000008
:1068b0001c1c00001c1c00001c1c00001c1d0000f7
:1068c0001d1d00001d1d00001d1e00001e1e0000dd
:1068d0001e1f00001f1f00001f1f00001b170000cd
:1068e000171300000f0b00000b070000030300004c
:1068f000032300004343000063a300008363000000
:10690000634300002323000003030000030700008b
:106910000b0b00000f130000171700001b1f0000d7
:106920001f1f00001f1f00001e1e00001e1e000073
:106930001e1d00001d1d00001d1d00001d1c00006f
:106940001c1c00001c1c00001c1c00001c1c000067
:106950001c1c00001c1c00001d1d00001d1d000053
:106960001d1d00001e1e00001e1e00001e1f000038
:106970001f1f00001f1f00001b170000171300003f
:106980000f0b00000b0700000303000003230000af
:106990002343000063630000a383000083630000bf
:1069a0004343000023230000030300000707000007
:1069b0000b0f00000f130000171b00001b1f00002f
:1069c0001f1f00001f1f00001e1e00001e1e0000d3
:1069d0001e1d00001d1d00001d1d00001d1d0000ce
:1069e0001d1d00001d1d00001d1d00001d1d0000bf
:1069f0001d1d00001d1d00001d1d00001d1d0000af
:106a00001e1e00001e1e00001e1f00001f1f000093
:106a10001f1f00001b1b0000171300000f0f0000ba
:106a20000b070000070300000323000023430000be
:106a30004363000083c30000a3830000836300005e
:106a400043230000230300000303000007070000a6
:106a50000b0f000013130000171b00001b1f00008a
:106a60001f1f00001f1f00001e1e00001e1e000032
:106a70001e1e00001e1d00001d1d00001d1d00002b
:106a80001d1d00001d1d00001d1d00001d1d00001e
:106a90001d1d00001d1d00001e1e00001e1e00000a
:106aa0001e1e00001e1f00001f1f00001f1f0000f1
:106ab0001b1b000017130000130f00000b07000042
:106ac00007030000030300002323000043630000ca
:106ad00083830000c3a30000a3830000634300007e
:106ae000432300002303000003030000070b000002
:106af0000b0f000013130000171b00001b1f0000ea
:106b00001f1f00001f1f00001f1e00001e1e000090
:106b10001e1e00001e1e00001e1d00001d1d000088
:106b20001d1d00001d1d00001d1d00001d1d00007d
:106b30001e1e00001e1e00001e1e00001e1e000065
:106b40001f1f00001f1f00001f1f00001b1b000055
:106b500017130000130f00000b0b000007030000c9
:106b6000030300002323000043430000638300006d
:106b7000a3c30000c3a3000083830000634300009d
:106b8000432300002303000003030000070b000061
:106b90000b0f000013130000171700001b1b000051
:106ba0001f1f00001f1f00001f1f00001e1e0000ef
:106bb0001e1e00001e1e00001e1e00001e1e0000e5
:106bc0001e1e00001e1e00001e1e00001e1e0000d5
:106bd0001e1e00001e1e00001e1f00001f1f0000c2
:106be0001f1f00001f1b00001b17000017130000d1
:106bf000130f00000b0b000007030000030300004d
:106c000023230000434300006383000083a30000ac
:106c1000e3c30000c3a300008383000063430000bc
:106c2000432300000303000003070000070b0000dc
:106c30000b0f000013130000171700001b1b0000b0
:106c40001f1f00001f1f00001f1f00001f1e00004d
:106c50001e1e00001e1e00001e1e00001e1e000044
:106c60001e1e00001e1e00001e1e00001e1e000034
:106c70001e1e00001f1f00001f1f00001f1f00001e
:106c80001f1b00001b17000017130000130f00004c
:106c90000b0b0000070700000303000003230000a4
:106ca000434300006383000083a30000c3e30000ac
:106cb000c3c30000a3a3000083630000634300007c
:106cc000232300000303000003070000070b00005c
:106cd0000b0f00000f130000171700001b1b000014
:106ce0001b1f00001f1f00001f1f00001f1f0000b0
:106cf0001f1e00001e1e00001e1e00001e1e0000a3
:106d00001e1e00001e1e00001e1e00001f1f000091
:106d10001f1f00001f1f00001f1f00001b1b000083
:106d20001b170000171300000f0f00000b0b0000d3
:106d300007070000030300000323000023430000b3
:106d40006363000083a30000a3c30000e3e300002b
:106d5000c3c30000a383000083630000434300001b
:106d6000232300000303000003070000070b0000bb
:106d70000b0f00000f13000013170000171b00007b
:106d80001b1b00001f1f00001f1f00001f1f000013
:106d90001f1f00001f1f00001f1f00001f1f0000fb
:106da0001f1f00001f1f00001f1f00001f1f0000eb
:106db0001f1f00001f1b00001b1b000017170000f7
:106dc000131300000f0f00000b0b0000070700005b
:106dd000030300000323000023430000436300007b
:106de00083830000a3c30000c3e30000e3e30000cb
:106df000c3c30000a383000083630000434300007b
:106e00002323000003030000030300000707000022
:106e10000b0b00000f1300001317000017170000e2
:106e20001b1b00001b1f00001f1f00001f1f000076
:106e30001f1f00001f1f00001f1f00001f1f00005a
:106e40001f1f00001f1f00001f1f00001f1f00004a
:106e50001b1b00001b170000171700001313000076
:106e60000f0b00000b0700000703000003030000e6
:106e700003230000234300004363000083830000da
:106e8000a3c30000c3e30000e3e30000e3e300006a
:106e9000c3c30000a38300008363000043430000da
:106ea0002323000003030000030300000707000082
:106eb0000b0b00000f0f000013130000171700004a
:106ec000171b00001b1b00001b1f00001f1f0000e2
:106ed0001f1f00001f1f00001f1f00001f1f0000ba
:106ee0001f1f00001f1f00001b1b00001b1b0000ba
:106ef0001717000017130000130f00000f0b0000fe
:106f00000b07000007030000030300000323000039
:106f1000234300004363000083830000a3c30000f9
:106f2000c3e30000e3e20000e3e30000e3c300008a
:106f3000c3a30000a3830000836300004343000059
:106f400023230000030300000303000007070000e1
:106f50000b0b00000b0f00000f13000013170000b5
:106f600017170000171b00001b1b00001b1b000055
:106f70001b1b00001b1b00001b1b00001b1b000039
:106f80001b1b00001b1b0000171700001717000039
:106f9000131300000f0f00000b0b00000b07000085
:106fa0000703000003030000032300002343000045
:106fb0004363000083830000a3a30000c3c3000059
:106fc000e3e30000e2e20000e3e30000e3c30000cb
:106fd000c3a30000a38300008363000043430000b9
:106fe0002323000023030000030300000307000025
:106ff000070b00000b0b00000f0f00001313000025
:10700000131700001717000017170000171b0000c8
:107010001b1b00001b1b00001b1b000017170000a0
:10702000171700001717000013130000130f0000bc
:107030000f0b00000b0b000007070000030300000c
:1070400003030000232300002343000043630000e8
:1070500083830000a3a30000c3c30000e3e3000098
:10706000e3e20000e2e30000e3e30000e3c300002a
:10707000c3a30000a3830000836300004343000018
:107080004323000023030000030300000307000064
:10709000070700000b0b00000b0f00000f0f000094
:1070a000131300001313000013170000171700003c
:1070b0001717000017170000171700001313000020
:1070c00013130000130f00000f0f00000b0b000044
:1070d0000b07000007070000030300000303000084
:1070e0002323000043430000436300008383000028
:1070f000a3a30000c3c30000e3e30000e3e3000038
:10710000e2e20000e2e30000e3e30000e3c300008a
:10711000c3a30000a3830000836300006343000057
:1071200043230000232300000303000003030000a7
:1071300007070000070b00000b0b00000b0f0000ff
:107140000f0f00000f0f00001313000013130000b7
:107150001313000013130000130f00000f0f0000a3
:107160000f0f00000b0b00000b0b000007070000c7
:107170000703000003030000032300002323000093
:10718000434300006363000083830000a3a3000067
:10719000c3c30000e3e30000e3e30000e2e100001a
:1071a000e2e20000e2e30000e3e30000e3c30000ea
:1071b000c3a30000a38300008363000063430000b7
:1071c0004323000023230000030300000303000007
:1071d0000307000007070000070b00000b0b00006f
:1071e0000b0b00000b0f00000f0f00000f0f000033
:1071f0000f0f00000f0f00000b0b00000b0b000027
:107200000b0b000007070000070700000303000046
:107210000303000003230000232300004343000076
:107220006363000083830000a3a30000c3c30000c6
:10723000e3e30000e3e30000e2e20000e1e100003c
:10724000e2e20000e2e30000e3e30000e3c3000049
:10725000c3c30000a38300008383000063430000d6
:107260004343000023230000230300000303000026
:1072700003030000030700000707000007070000e2
:107280000b0b00000b0b00000b0b00000b0b0000a6
:107290000b0b00000b0b00000b07000007070000a2
:1072a00007070000030300000303000003030000be
:1072b00023230000234300004343000063830000b6
:1072c00083830000a3c30000c3c30000e3e3000006
:1072d000e3e30000e2e20000e2e10000e1e100009f
:1072e000e2e20000e2e30000e3e30000e3c30000a9
:1072f000c3c30000a3a300008383000063630000f6
:107300004343000043230000232300000303000045
:10731000030300000303000003030000070700004d
:107320000707000007070000070700000707000025
:107330000707000007070000070300000303000021
:1073400003030000030300000323000023230000c5
:1073500043430000436300006383000083a30000f5
:10736000a3c30000c3c30000e3e30000e3e30000a5
:10737000e2e20000e2e10000e1e10000e1e1000002
:10738000e2e20000e2e30000e3e30000e3c3000008
:10739000c3c30000a3a30000838300008363000035
:1073a0006343000043430000232300002323000025
:1073b00003030000030300000303000003030000b5
:1073c00003030000030300000303000003030000a5
:1073d0000303000003030000030300000303000095
:1073e0000323000023230000234300004343000045
:1073f000636300008383000083a30000a3c3000035
:10740000c3c30000e3e30000e3e30000e2e20000a6
:10741000e2e10000e1e00000e1e10000e1e1000064
:10742000e2e20000e2e30000e3e30000e3e3000047
:10743000c3c30000c3a30000a38300008363000054
:107440006363000043430000432300002323000044
:1074500023230000030300000303000003030000d4
:107460000303000003030000030300000303000004
:107470000303000003030000032300002323000094
:1074800023230000434300004363000063630000c4
:1074900083830000a3a30000c3c30000c3e3000074
:1074a000e3e30000e3e30000e2e20000e2e10000c9
:0474b000e1e1000016
:020000040000fa
:1074b4001000fa005007980061079800624f980086
:1074c400734f9800de029000e4042000848f520081
:1074d4004e013e00ee029000e41d2000848f520015
:1074e4004c013e000002eb00140798003201370003
:1074f4000002eb00040f7800190137006e4a900077
:107504000482fb00cfa2de006a2bb90006037800d8
:107514006020b900800378000703430084027800e8
:10752400a4002000042ab800050343008602780062
:1075340066024200e0824a00a6b62000060242002b
:107544001400be006e4a90000482fb00cfa2de004d
:107554006a2bb900060378006021b9008203780021
:107564000703430084027800a4002000042ab80022
:107574000503430086027800a6b6200006024200f6
:10758400144278008482fb001e02900004aab90011
:10759400040278001e02420005002000040240009c
:1075a400858248009601800004f0a4008582d20000
:1075b4009501880014427800444798009601880099
:1075c4006e4a90000482fb00cfa2de006a2bb90051
:1075d400060378006020b9008003780007034300a5
:1075e40084027800a4002000042ab80005034300a4
:1075f4008602780062024200e0824a00a6b62000b9
:1076040006024200944290004e42900084cf520001
:10761400bf0032004e4290000482fb000400780058
:10762400e30a07007e4a90000482fb00cfa2de003a
:107634003600200007002000860f5200878f5a0072
:10764400b5003e0004600100030037002600370047
:1076540064003700b20037005e0290001e02420050
:10766400340798001e029000c222dd006e029000d2
:10767400848242001e0290000402420004824200fe
:1076840044079800be029000d4042000848f520066
:10769400a5003e004e0290006123b80084cb200078
:1076a400144278000482fb0005002000001e200024
:1076b400010020000402500085825800840f53000a
:1076c400858f5b00d50031004e029000050020003c
:1076d4003e039000070020000401be000600be0027
:1076e400d10007009d0037006e4a90000482fb0021
:1076f400cfa2de006a2bb900060378006020b9002f
:10770400800378000703430084027800a40020006b
:10771400042ab8000503430086027800a6b62000b8
:1077240006024200144278008482fb001e0290008c
:10773400848252005e029000048242000402e90046
:107744003407980084cb2000144278008482fb0024
:107754001e02780004aab900840278006e02900028
:107764000482420044079800be029000e404200012
:10777400848f52006e003e003e029000e00f5200e3
:107784006d0032004e0290006123b80084cb2000cb
:10779400144278000482fb0005002000001e200033
:1077a400010020000402500085825800840f530019
:1077b400858f5b00620031004e029000e00f5200a2
:1077c400610032004e029000050020003e0390004c
:1077d400070020000401be000600be00920007005e
:1077e4005e0037006e4a90000482fb00cfa2de00e8
:1077f4006a2bb900060378006020b9008003780082
:107804000703430084027800a4002000042ab8007f
:107814000503430086027800a6b620000602420053
:10782400144278000482fb009e0252005e02900023
:10783400048242000402e9003407980084cb20004b
:10784400144278000481fb006e4a90000482fb001d
:10785400cfa2de006a2bb900060378006020b900cd
:10786400800378000703430084027800a40020000a
:10787400042ab8000503430086027800a6b6200057
:1078840006024200144290008482fb001e02900013
:10789400048252000402e9000492b90084027800d0
:1078a4006e0290000482420044079800be029000d9
:1078b400e4042000848f520025003e004e02900014
:1078c4006123b80084cb2000144278000482fb00ba
:1078d40005002000001e20000100200004025000ca
:1078e40085825800840f5300858f5b001a00310095
:1078f4004e029000050020003e0390000700200087
:107904000401be000600be00470007001300370054
:107914000000000011003700000000000f003700d5
:10792400000000000d003700000000000b003700cd
:1079340000000000090037000000000007003700c5
:1079440000000000050037000000000003003700bd
:107954000000000001003700000000001e0fe800d6
:107964006e4a90000482fb00cfa2de006a2bb900ad
:10797400060378006020b900800378000703430001
:1079840084027800a4002000042ab8000503430000
:1079940086027800a6b6200006024200144278004f
:1079a4000482fb009e0f5200d4fe3e001e02900093
:1079b4000402e800140798006e4a90000482fb0059
:1079c400cfa2de006a2bb900060378006020b9005c
:1079d400800378000703430084027800a400200099
:1079e400042ab8000503430086027800a6b62000e6
:1079f40006024200144290008482fb001e029000a2
:107a0400848f5200bafe3e000500370000000000db
:107a140003003700000000000100370000000000f0
:107a24000080fa00000006000800fa00008fbe0083
:107a34002207980033079800be0290000405200036
:107a440004aab900040378002e0290006022b90051
:107a54000402780004034300ae02900004052000f1
:107a6400042ab80005034300860278001e0f420072
:107a74005e974a000000000001003700000000008b
:107a84003438800062026200e00f5200fbff3a00cb
:107a94001e027800043888001e02be00402ade0060
:107aa400840278000430260005027200143888002d
:107ab400000000000100370000000000343880009e
:107ac40062026200e00f5200fbff3a0064002100f2
:107ad40004388800044026001438880000000000a0
:107ae40001003700000000003438800062026200a8
:107af400e00f5200fbff3a0004062000043888001f
:107b04000470260014388800000000000080fa0089
:107b1400000006000800fa002007980031079800ca
:107b2400ae029000f4042000848f5200020036005c
:107b3400f40420002407980084cb20001442780029
:107b44008482fb002e02900004aab900840278000b
:107b5400f41d2000848f520002003600f41d200022
:107b6400240798002e0290000402d1008502200010
:107b740004825200040f780084cb20001442780061
:107b84008482fb002e02900004aab900040278004b
:107b94000402d100050f200004825200140798004b
:107ba4009e027800e4042000848f52001a003e00f4
:107bb4009e029000e41d2000848f520018003e00b5
:107bc4001e027800e00f5200170034001e029000dd
:107bd400e00f5200160034003e00900074090700c4
:107be40084cb2000144278008482fb002e02900093
:107bf40004aab900040378009e0290001e027800d3
:107c0400860178002e019000850078000400780039
:107c14008d09070007003700000000000500370049
:107c240000000000030037000000000001003700de
:107c3400000000000080fa00000006000a00fa00bc
:107c440040079800140020002407980084cb2000eb
:107c5400144278000482fb000402420034079800b6
:107c6400be029000e4042000848f52002c003e00e9
:107c7400ae029000e41d2000848f52002a003e00d2
:107c84003e029000e00f5200290032002e029000c4
:107c9400e00f5200280032000002eb00040f7800cd
:107ca4001a0037000002eb00140798001100370097
:107cb4004e0290009e0242001e0290000482420086
:107cc400f4648800f4648000040078003809070034
:107cd400be0190002e0190009e0078001e009000ce
:107ce400590907009e0290002e029000048242006f
:107cf400140798009e029000e4042000848f520030
:107d0400ebff36003e0290001e0f4200e41d2000ef
:107d14009e027800848f5200e2ff3600070037008d
:107d240000000000050037000000000003003700d9
:107d34000000000001003700000000000080fa008d
:107d4400000006000200fa00000f780015cb2000a6
:107d54009542780004cb2000144278001e0378007a
:107d6400064378008641780002c72000f1c620004f
:107d7400e0c620006f0b070006c7200016437800fa
:107d8400f5c6200095427800e4c62000144278002d
:107d94000641780085407800044078002f0b0700e6
:107da400004278000482fb00f4648800346480009c
:107db400d464880044648000e4648800956580008d
:107dc4007464800004aab9008402780034648000da
:107dd4000482420034648800a565800084648000c5
:107de40004aab9008402780044648000048242003a
:107df4004464880035648000b4648000848f520039
:107e040005003400b4648000346488009465800004
:107e14000402ea009465880045648000c46480001c
:107e2400848f520005003400c464800044648800d8
:107e3400a46580000402ea00a4658800356480001b
:107e440094648000848f520005003c009464800098
:107e540034648800946580000402ea009465880014
:107e640045648000a4648000848f520005003c00b7
:107e7400a464800044648800a46580000402ea00cd
:107e8400a46588000000eb00c90807006464800052
:107e9400840378005464800004037800e464800060
:107ea40084027800d4648000870178000601780099
:107eb4008500780004007800e3080700f46480007b
:107ec40004007800ba080700646480008403780022
:107ed40054648000040378004464800084027800c1
:107ee40034648000870178000601780085007800fa
:107ef40004007800d408070044648000cfa2de00a8
:107f040036648000cfb3de000401be000600be006c
:107f1400c5fe07000080fa00000006001000fa0009
:107f24007007980000c2eb006447980000c2eb00a1
:107f340074479800840220002407980084cb200012
:107f4400144278008482fb002403200004aab900b0
:107f540004027800040f78003b0037007e02900092
:107f64000442780004424200844278002e029000c9
:107f7400044278000414a20084c052006c0047003c
:107f8400eb0347006a034700fe4290006e429000f4
:107f940081417800000178008700780006007800ad
:107fa400e40a07004e4b9000be4a90002e4a90000f
:107fb400064178008540780004407800a70a07004d
:107fc400004278000482fb00440798004e009000b1
:107fd400770807002e0290000482e9002407980025
:107fe4002e029000e00f520002003d000002eb0060
:107ff400240798000002eb00140798000a003700d9
:108004001e027800050020001e03900007002000d7
:108014000401be000600be0083fe07001e0290009d
:108024000402e800140798009e029000e404200073
:10803400848f5200f2ff360084cb20001442780073
:108044000482fb001e0f42001e0278006123b80068
:1080540084cb2000144278000482fb000500200039
:10806400001e2000010020000402500085825800f8
:10807400840f5300858f5b00b8ff39000080fa003d
:10808400000006000200fa00000f78001e007800cd
:10809400a2ff07001e0278000442780063426200d7
:1080a40068434200b4bb2000144278008482fb0081
:1080b40084cb2000144278000482fb0004aab90097
:1080c4008402780024002000110009008402d800f2
:1080d400000278008516200084825200a4bb200090
:1080e400144278000482fb000402d10004427800a8
:1080f4000482fb0027042000048253008041eb002b
:10810400064178008500780004007800e8fc070048
:10811400c200200003002000e1ea280020c720005c
:1081240000e40700d21420008000eb0020c72000e8
:10813400d10d07000201200003002000a1eb28005c
:1081440020c72000f7e30700221620008000eb0080
:1081540020c72000c80d0700d20020000300200023
:10816400a1ec280020c72000eee3070072172000ce
:108174008000eb0020c72000bf0d0700646480006e
:10818400c512200004825200c46488001e007800d6
:10819400ecfe07000080fa00000006000400fa006c
:1081a400100798000002eb00040f78001e0078000e
:1081b4005aff07001e0278000442780063426200fe
:1081c40068434200b4bb2000144278008482fb0060
:1081d40084cb2000144278000482fb0004aab90076
:1081e4008402780024002000110009008402d800d1
:1081f400000278008516200084825200a4bb20006f
:10820400144278000482fb000402d1000442780086
:108214000482fb0027042000048253008041eb0009
:10822400064178008500780004007800a0fc07006f
:10823400e20020000300200071ed280020c7200088
:10824400b8e30700d21420008000eb0020c7200010
:10825400890d0700f20020000300200051ee2800e1
:1082640020c72000afe30700221620008000eb00a7
:1082740020c72000800d07000080fa0000000600df
:108284000000fa00140020005464880084cb20000d
:10829400144278000482fb00646488005464800003
:1082a4007464880064648000846488000002eb00c5
:1082b400946488000002eb00a46488005464800085
:1082c400f504200004825200b464880064648000d1
:1082d400c512200004825200c46488000080fa00a1
:1082e400000006000200fa00000f780064648000b9
:1082f400051e200004825200c46488001e00780019
:1083040090fe070084cb2000144278000482fb0016
:108314008041eb0042c0b3008400780010002000cc
:1083240063fc0700320120000300200041ef280015
:1083340020c720007be30700d21420008000eb005c
:1083440020c720004c0d0700d200200003002000ad
:1083540071f0280020c7200072e3070022162000d5
:108364008000eb0020c72000430d07000080fa00c6
:10837400000006000000fa00f200200003002000c4
:1083840041f1280020c7200066e30700520a2000bc
:108394008000eb0020c72000370d070002012000f9
:1083a4000300200031f2280020c720005de307000d
:1083b400a20b20008000eb0020c720002e0d070038
:1083c400020120000300200031f3280020c7200010
:1083d40054e30700420e20008000eb0020c7200079
:1083e400250d0700f20020000300200031f42800ce
:1083f40020c720004be30700920f20008000eb0011
:1084040020c720001c0d07002201200003002000cb
:1084140021f5280020c7200042e30700e2102000d5
:108424008000eb0020c72000130d0700320120005c
:108434000300200041f6280020c7200039e307008c
:10844400821320008000eb0020c720000a0d0700e3
:10845400020120000300200071f7280020c720003b
:1084640030e30700221620008000eb0020c7200024
:10847400010d0700920020000300200071f828007d
:1084840020c7200027e30700721720008000eb00bc
:1084940020c72000f80c07000080fa000000060046
:1084a400849fbe00861f78003200f800042020005c
:1084b400940188000000fa0014658000e30f520064
:1084c4000e003a0044ca2000144278000482fb00e3
:1084d400cfa2de00669d2800040243001442780007
:1084e4000482fb004222de00044278000482fb0086
:1084f4004822dd00541688001e00370014658000f1
:10850400e10f52000e003a0044ca200014427800e1
:108514000482fb00cfa2de00e6ac28000402430084
:10852400144278000482fb004222de0004427800f8
:108534000482fb004822dd00541688000d00370039
:1085440044ca2000144278000482fb00cfa2de005b
:10855400668d280004024300144278000482fb0064
:108564004222de00044278000482fb004822dd003f
:108574005416880044ca2000144278000442e800db
:108584000443780045ca2000864a78008460a90024
:108594000080fa003200f9004f0378004f02be0059
:1085a400004006000000fa0005658000b42b20009e
:1085b400848f520003003e000002eb001465880023
:1085c4002200370005658000f4312000848f5200ba
:1085d40003003e0024002000146588001b003700bf
:1085e4000565800034512000848f520003003e0052
:1085f40034002000146588001400370005658000ed
:10860400b45d2000848f520003003e00140020005b
:10861400146588000d00370005658000349c200037
:10862400848f520003003e0044002000146588003b
:108634000600370005658000449c2000848f5200aa
:10864400020036000002eb00046588001465800017
:10865400050020004600200007002000860f52007d
:10866400878f5a001f003e00046001000400370099
:10867400080037000c0037001000370014003700e2
:1086840031e7a900046580000400780015ff0700a5
:108694001700370031e7a800046580000400780063
:1086a40066fd07001200370031e7a9000465800069
:1086b40004007800b9fe07000d00370031e7a90077
:1086c40004658000040078006efe0700080037008f
:1086d40031e7a900046580000400780025ff070045
:1086e400030037000465800004007800fdfe0700e5
:1086f4000080fa00000006000000fa00a90b070041
:10870400a8ff07000000eb00a9060700031e2000d5
:10871400120020008000eb00f0042000ca060700cd
:108724007b0b0700046580000402e80004658800f0
:10873400f2ff37000000fa00889fbe008a9fbe0047
:108744000002eb00142788000002eb0024278800b5
:108754000002eb00342788000002eb005427880055
:108764000002eb00642788000002eb004416880036
:108774000a87a9000887a800a080a8009d0a07000e
:1087840038080700fd0b0700800c0700c20707002c
:10879400dd030700bafe07000ac025000b00200015
:1087a4000a00be0091060700bb07070008c02500a9
:1087b4000900200004602100150020000803d000f7
:1087c4008403d000070243004220a80085824c00a5
:1087d4004200a9004220ae004200a8000482d30057
:1087e4000400be0081060700ab070700c2ff0700b4
:1087f4000002eb00040078004f05be004f04be00e9
:088804000080fa0000000600ec
:020000040000fa
:10880c006e0c00003800000080000000b00c00006e
:10881c000800000082000000ffff010000010000c2
:10882c0001000000b80c00000200000082000000f3
:10883c0006000000005c0000002c0000800000001e
:10884c000008000000020000800000006a0b00001d
:10885c008400000080000000000a00006a01000093
:10886c0080000000ee0b0000800000008200000081
:10887c009101dd0001910100dd01650001dd0100c8
:10888c006501dd00013e0100dd013e0001dd01005e
:10889c003e01dd0001c201006501910001dd010016
:1088ac009101dd0001650100dd01650001dd0100c4
:1088bc003e01dd00013e0100dd013e0001dd010055
:1088cc003e012c0001910100dd01910001dd010050
:1088dc006501dd0001650100dd013e0001dd0100e7
:1088ec003e01dd00013e0100dd01fd0000ee000057
:1088fc009f00ee00003e0100dd019f0000ee000035
:10890c0065012c00019f0000ee00b20000ee00009b
:10891c009101dd0001d40000c8000000ba0c000079
:10892c000200000080000000bc0c000002000000ef
:10893c0080000000be0c000002000000820000005d
:10894c00cb010000ac520000540900008200000072
:10895c0000002000007e00001500040084010000cf
:10896c00029901000005ae0001000500c3010000e2
:10897c0005d801000005ed00010005000202000011
:10898c000217020000052c00020005004102000045
:10899c000556020000056b00020002008002000078
:1089ac00059502000002aa0002000500bf020000ab
:1089bc0005d402000002e90002000500fe020000de
:1089cc000513030000052800030005003d0300000b
:1089dc000552030000056700030005007c0300003e
:1089ec00059103000002a60003000200bb03000077
:1089fc0005d003000005e50003000500fa030000a4
:108a0c00040f0400000524000400040039040000d5
:108a1c00044e040000046300040004007804000009
:108a2c00048d04000004a20004000400b70400003c
:108a3c0004cc04000002e10004000400f604000071
:108a4c00040b05000004200005000600350500009d
:108a5c00044a050000045f000500040074050000d2
:108a6c000489050000049e0005000400b305000005
:108a7c0004c805000004dd0005000400f205000038
:108a8c000607060000041c00060004003106000066
:108a9c000446060000055b00060005007006000099
:108aac000585060000059a0006000500af060000cb
:108abc0003c406000004d90006000400ee06000002
:108acc000403070000041800070004002d07000031
:108adc000442070000045700070004006d07000063
:108aec00028207000004970007000400ad07000095
:108afc0002c207000006d70007000400ec070000c4
:108b0c000401080000041600080004002c080000f2
:108b1c000442080000045700080003006c08000021
:108b2c00048108000004960008000600ab08000051
:108b3c0004c008000004d50008000400eb08000085
:108b4c000500090000021500090005002a090000b3
:108b5c00063f0900000000000000000000000000bb
:108b6c0000000000000000000000000000000000f9
:108b7c0000000000000101000101010001010100e1
:108b8c0001010100010001000000000000000000d4
:108b9c0000000000000005000500000000000000bf
:108bac0000000000000000000000000000000000b9
:108bbc000000000005050700050505000705050078
:108bcc000000000000000000000000000000020097
:108bdc000705010007070400050507000200000057
:108bec00000000000000000000000000050404006c
:108bfc00020202000101050000000000000000005c
:108c0c000000000000000000020502000505050040
:108c1c000505070004000000000000000000000033
:108c2c000000010001000000000000000000000036
:108c3c000000000000000000000000000402020020
:108c4c000101010001010100010102000204000008
:108c5c0000000000000000000102020004040400f7
:108c6c0004040400040402000201000000000000df
:108c7c0000000000000207000200000000000000dd
:108c8c0000000000000000000000000000000000d8
:108c9c0000000000000002000707020000000000b6
:108cac0000000000000000000000000000000000b8
:108cbc0000000000000000000000010001000000a6
:108ccc000000000000000000000000000000000098
:108cdc00070700000000000000000000000000007a
:108cec000000000000000000000000000000000078
:108cfc000000010000000000000000000000000067
:108d0c00000404000404020002020200020101003b
:108d1c000101000000000000000707000505050028
:108d2c000505050005050500050507000000000008
:108d3c00000000000001010001010100010101001f
:108d4c000101010001010100000000000000000011
:108d5c0000070700040407000101010001010100e4
:108d6c0001010700000000000000000000070700e0
:108d7c0004040700040404000404040004040700b1
:108d8c0000000000000000000005050005050700bc
:108d9c0004040400040404000404040000000000a3
:108dac000000000000070700010107000404040094
:108dbc00040404000404070000000000000000008c
:108dcc000007070001010700050505000505050062
:108ddc000505070000000000000000000007070068
:108dec000404040004040400040404000404040047
:108dfc000000000000000000000707000505070048
:108e0c000505050005050500050507000000000027
:108e1c00000000000007070005050700040404001b
:108e2c00040404000404070000000000000000001b
:108e3c000000000000000000010000000000000025
:108e4c000000010000000000000000000000000015
:108e5c000000000001000000000000000000010004
:108e6c0001000000000000000000000000000000f5
:108e7c0000040200010302000400000000000000d6
:108e8c0000000000000000000000000000000700cf
:108e9c0000070700000000000000000000000000b8
:108eac0000000000000000000001020004060200a7
:108ebc000100000000000000000000000007070097
:108ecc000504060002020200020202000200020077
:108edc000000000000000000000707000507050067
:108eec000505050005050500070107000000000049
:108efc000000000000070700050507000505050038
:108f0c000505050005050500000000000000000037
:108f1c00000707000505030005050500050505000c
:108f2c000505070000000000000000000007070016
:108f3c00050101000101010001010100010507000b
:108f4c000000000000000000000303000505050000
:108f5c0005050500050505000505030000000000da
:108f6c0000000000000707000501070001010100d7
:108f7c0001010100010507000000000000000000d5
:108f8c0000070700010107000101010001010100b8
:108f9c0001010100000000000000000000070700b4
:108fac00050101000101010005050500050507008b
:108fbc00000000000000000000050500050507008a
:108fcc000505050005050500050505000000000068
:108fdc00000000000001010001010100010101007d
:108fec00010101000101010000000000000000006f
:108ffc000004040004040400040404000404040039
:10900c000505070000000000000000000005050039
:10901c00050503000505050005050500050505000a
:10902c00000000000000000000010100010101002f
:10903c000101010001010100010107000000000015
:10904c0000000000001f1f00151515001515150058
:10905c001515150015151500000000000000000086
:10906c0000070700050505000505050005050500b9
:10907c0005050500000000000000000000070700c7
:10908c000505050005050500050505000505070096
:10909c0000000000000000000007070005050500a7
:1090ac00050505000507070001010100000000008f
:1090bc000000000000070700050505000505050078
:1090cc000505050005050700020200000000000070
:1090dc00000707000505030005050500050505004b
:1090ec000505050000000000000000000007070057
:1090fc000501070004050500050505000505070029
:10910c00000000000000000000070700020202003f
:10911c000202020002020200020202000000000031
:10912c00000000000005050005050500050505000b
:10913c000505050005050700000000000000000003
:10914c0000050500050505000505050005050500dc
:10915c0005050200000000000000000000151500cd
:10916c0015151500151515001515150015151a00f2
:10917c0000000000000000000005050005050200cd
:10918c0005050500050505000505050000000000a6
:10919c0000000000000505000505020002020200a7
:1091ac0002020200020202000000000000000000a7
:1091bc00000707000404040002020200020301007d
:1091cc00010107000000000000000000000000008a
:1091dc000701010001010100010101000101010071
:1091ec000107000000000000000101000101010066
:1091fc000202020002060400040404000000000045
:10920c000000000000000000070404000404040037
:10921c00040404000404040004070000000000001f
:10922c00000000000002050000000000000000002b
:10923c000000000000000000000000000000000022
:10924c000000000000000000000000000000000012
:10925c0000070000000000000000000000000100fa
:10926c0002000000000000000000000000000000f0
:10927c0000000000000000000000000007050400d2
:10928c0007070500050507000000000000000000ae
:10929c00000101000101010007050500050505009d
:1092ac0005050700000000000000000000000000a1
:1092bc00000000000701010001010100010107008d
:1092cc00000000000000000000040400040404007e
:1092dc000705050005050500050507000000000051
:1092ec000000000000000000000000000701010069
:1092fc00070701000101070000000000000000004a
:10930c000000000000000000070101000707010039
:10931c00010101000000000000000000000000003e
:10932c000000000007050500050505000505070000
:10933c000404040007070000000001000101010003
:10934c0001070500050505000505050005000000e1
:10935c0000000000000000000000010000010100fe
:10936c0001010100010101000100000000000000ea
:10937c0000000000000004000004040004040400c9
:10938c0004040400040404000407070000000000a7
:10939c000101010001010500050503000705050099
:1093ac0005050000000000000000000001010100a4
:1093bc000101010001010100010101000101000096
:1093cc0000000000000000000000000000001f0072
:1093dc0015151500151515001515000000000000d9
:1093ec00000000000000000000000700050505005b
:1093fc000505050005050000000000000000000048
:10940c00000000000000070005050500050505002b
:10941c000507000000000000000000000000000034
:10942c0000000700050505000505050005070100fe
:10943c00010101000100000000000000000000001c
:10944c0007050500050505000505070004040400d3
:10945c0004040000000000000000000000070500ec
:10946c0001010100010101000100000000000000e9
:10947c0000000000000000000007050001070700c5
:10948c0004050500070000000000000000000100ba
:10949c0001010100010301000101010001010100b2
:1094ac0003000000000000000000000000000000ad
:1094bc000005050005050500050505000700000071
:1094cc000000000000000000000000000005050086
:1094dc000505050005050500020000000000000060
:1094ec000000000000000000001515001515150007
:1094fc00151515001a000000000000000000000007
:10950c000000000000050500050207000505050028
:10951c00050000000000000000000000000000003a
:10952c0000050500050505000505050007040400f8
:10953c000407070000000000000000000000070006
:10954c0004040200020201000107000000000000f8
:10955c0000000000000004000202020002020100f0
:10956c0003020200020202000400000000000000de
:10957c0001010100010101000101010001010100d3
:10958c0001010100010100000000000000000100c9
:10959c0002020200020204000602020002020200a1
:1095ac0001000000000000000000000000000000ae
:1095bc00001a05000500000000000000000000007b
:1095cc00a60c00000a00000080000000c00c000087
:1095dc00020000008200000001000000c20c00002c
:1095ec000200000080000000c80c00000200000017
:1095fc0080000000c40c000004000000800000008b
:04960c00000000005a
:020000040000fa
:109610000c00fa00008fbe00220798003307980064
:1096200044079800550798001e02be000402780007
:10963000643888001e02be00040278007438880076
:109640002e029000be029000040278008438880048
:109650002e029000be029000040278009438880028
:1096600000000000010037000000000034388000d6
:1096700062026200e00f5200fbff3a000002eb00c2
:109680000438880004102700143888000000000007
:1096900000000000010037000000000034388000a6
:1096a00062026200e00f5200fbff3a000002eb0092
:1096b00004388800042027001438880000000000c7
:1096c0000000000001003700000000003438800076
:1096d00062026200e00f5200fbff3a004e0290006f
:1096e000043888004e029000de029000402ade001e
:1096f00084027800044027000502720014388800b4
:10970000000000000080fa00000006001000fa00cf
:10971000889fbe008a9fbe008c9fbe000002eb00a7
:10972000140798000002eb00040f7800e0003700f7
:109730001e0290006123b80008f9200009102000e3
:109740000802be000402430085824b00960180009f
:1097500004f0a4008582d20095018800944078002e
:10976000960188001e0278006123b8006a3ab900a9
:10977000040078006032b900040278000400400060
:1097800086027800a4002000042ab80005004000ea
:1097900080027800a6b6200006024200014a780046
:1097a0001e0290000402e8006123b8000af92000bc
:1097b0000b1020000a02be000402430085824b0009
:1097c0009601800004f0a4008582d20095018800f3
:1097d00094407800960188001e0278006123b8004a
:1097e0006a3ab900040078006032b90004027800d7
:1097f0000400400086027800a4002000042ab8007b
:109800000500400080027800a6b620000602420053
:10981000114298001e0290000482e8006123b80003
:109820000cf920000d1020000c02be0004024300c1
:1098300085824b009601800004f0a4008582d2004e
:109840009501880094407800960188001e027800f7
:109850006123b8006a3ab900040078006032b900a8
:10986000040278000400400086027800a400200072
:10987000042ab8000500400080027800620342001c
:10988000e0834a00a4b6200004024300014a7800a5
:109890001e029000630242006123b80004f9200018
:1098a0002407980004102000340798002e0290002e
:1098b000be0290000402430085824b0096018000a6
:1098c00004f0a4008582d2009501880094407800bd
:1098d000960188001e0278006123b8006a3ab90038
:1098e000040078006032b9000402780004004000ef
:1098f00086027800a4002000042ab8000500400079
:109900008002780062034200e0834a00a4b620008f
:1099100004024300114298001e02900064024200bb
:109920006123b80004f920004407980004102000c7
:10993000540798004e029000de029000040243009b
:1099400085824b009601800004f0a4008582d2003d
:109950009501880094407800960188001e027800e6
:109960006123b8006a3ab900040078006032b90097
:10997000040278000400400086027800a400200061
:10998000042ab80005004000800278006403420009
:10999000e0834a00a4b6200004024300014a780094
:1099a0001e029000650242006123b80004f9200005
:1099b0006407980004102000740798006e0290005d
:1099c000fe0290000401430085814b001e027800d6
:1099d0006123b8006a3ab900040078006032b90027
:1099e000040278000400400086027800a4002000f1
:1099f000042ab80005004000800278006603420097
:109a0000e0834a00a4b6200004024300028abe009c
:109a10001e0278006123b8006a3ab9000400780099
:109a20006032b90004027800040040008602780029
:109a3000a4002000042ab80005004000800278003d
:109a4000a6b6200006024200144278008480fb0083
:109a50001e0278006123b8006a3ab9000400780059
:109a60006032b900040278000400400086027800e9
:109a7000a4002000042ab8000500400080027800fd
:109a8000a6b6200006024200144290000482fb00a9
:109a9000048ab90004027800840278001e02900053
:109aa0000482420065024200140798001e0fe8007d
:109ab0001e027800ec0f52001dff36004f06be005c
:109ac0004f05be004f04be000080fa0000000600f3
:109ad0000800fa00881f7800008fbe002207980057
:109ae0003307980018c0b3002e019000be0190000b
:109af0001e00be0097db070000027800e00f520056
:109b000001003d000044eb00e04f54000a00320029
:109b10002e019000be0190001e00be00ebda07008f
:109b20000002be000400be008cdb07000002be0085
:109b300004027800090037001e01be002e009000cc
:109b4000be009000e1da07000002be000400be0083
:109b500082db07000002be000402780004007800e7
:109b60004f0478000080fa00000006002400fa008c
:109b7000889fbe008a1f7800500f9800610f9800e0
:109b8000625f980004179800151798000e10900057
:109b90009e10900087dc07000002be00240798009a
:109ba000350798000e1090009e10900025db0700ee
:109bb0000002be0044079800550798000002eb0021
:109bc000140798001e0137000002eb00040f780014
:109bd000050137006e5a90000482fb00cfa2de0020
:109be0006a2bb900060378006020b9008003780072
:109bf0000703430084027800a4002000042ab80070
:109c0000050343008602780066024200e0824a00b3
:109c1000a6b62000060242001400be006e5a900054
:109c20000482fb00cfa2de006a2bb9000603780095
:109c30006021b900820378000703430084027800a2
:109c4000a4002000042ab80005034300860278001f
:109c5000a6b6200006024200144278008482fb006f
:109c60001e02900004aab900040278001e024200fd
:109c70000500200004024000858248009601800013
:109c800004f0a4008582d200950188001442780077
:109c9000444f9800960188006e5a90000482fb00a1
:109ca000cfa2de006a2bb900060378006020b9005d
:109cb000800378000703430084027800a40020009a
:109cc000042ab800050343008602780062024200bd
:109cd000e0824a00a6b620000602420094429000ac
:109ce0004e4a900084cf5200b50032004e4a900098
:109cf0008482fb00645f80000482420004007800dc
:109d00002c0107006e5a90000482fb00cfa2de00f7
:109d10006a2bb900060378006020b9008003780040
:109d20000703430084027800a4002000042ab8003e
:109d30000503430086027800a6b620000602420012
:109d4000144278000482fb000402d100044278002f
:109d50000482fb001e021200740798006e5a9000e5
:109d60000482fb00cfa2de006a2bb9000603780054
:109d70006020b90080037800070343008402780064
:109d8000a4002000042ab8000503430086027800de
:109d9000a6b6200006024200144290000482fb0096
:109da0000402d100044278008482fb001e0290006d
:109db00004825200040f98007e029000cfa2de00c1
:109dc0000400be0006db07000002be004e0190004a
:109dd000de0190000400be0059db07000002be0057
:109de0000404be000e0a9000cfa2de000400be00f4
:109df000fbda07000002be002e019000be019000b9
:109e00000400be004edb07000002be000401be00dd
:109e10000800be002dda07000002be000400be00ec
:109e2000ceda07000002be00140f98007e029000f8
:109e3000cfa2de000400be00e9da07000002be0087
:109e40002e019000be0190000400be003cdb070024
:109e50000002be000404be000e0a9000cfa2de0085
:109e60000400be00deda07000002be004e019000d2
:109e7000de0190000400be0031db07000002be00de
:109e80000401be000800be0011da07000002be0097
:109e90000400be00b1da07000002be00240f9800e3
:109ea0001e0a9000cfa2de000400be00ccda07003c
:109eb0000004be007e029000cfa2de000400be00bf
:109ec000c7da07000002be000801be000400be00a1
:109ed000fffe070000027800840278005e0a90000e
:109ee00004824200340f980084cb20001442780092
:109ef0000485fb002e0a9000cfa2de000400be0005
:109f0000b7da07000004be000e0a9000cfa2de0000
:109f10000400be00b2da07000002be000801be0065
:109f20000400be00eafe07000002780004d2b90077
:109f300004027800840278006e0a900004824200d5
:109f4000440f9800be0a9000e4042000848f520061
:109f50001d003e003e0a9000e00f52001c0032003f
:109f60004e0a90006123b80084cb20001442780090
:109f70000482fb0005002000001e200001002000dc
:109f80000402500085825800840f5300858f5b00c7
:109f9000110031004e0a9000e00f52001000320014
:109fa0004e0a9000050020003e0b900007002000a4
:109fb0000401be000600be009cf607000900370041
:109fc0000000000007003700000000000500370017
:109fd000000000000300370000000000010037000f
:109fe000000000001e0fe8006e5a90000482fb0083
:109ff000cfa2de006a2bb900060378006020b9000a
:10a00000800378000703430084027800a400200046
:10a01000042ab8000503430086027800a6b6200093
:10a0200006024200144278000482fb009e0f520098
:10a03000e8fe3e001e0290000402e80014079800ab
:10a040006e5a90000482fb00cfa2de006a2bb9009a
:10a05000060378006020b9008003780007034300fe
:10a0600084027800a4002000042ab80005034300fd
:10a0700086027800a6b62000060242001442900034
:10a080008482fb001e029000848f5200cefe3e00b0
:10a090004f0578004f04be000080fa000000060063
:10a0a0000200fa00000f78001e0278000500200070
:10a0b0000400be004dda07000002be0002fd2000d1
:10a0c000930424000400be009dda07000002be00d5
:10a0d00002002000433324000400be00dbd9070047
:10a0e0000002be000400be000080fa00000006006e
:10a0f0001000fa00889fbe00008fbe002207980063
:10a1000033079800440798005507980066079800a1
:10a11000770798002e019000be0190001e00be003f
:10a120006ad907000002be000404be006e01900060
:10a13000fe0190003eb89700ceb8970063d90700a3
:10a140000002be000401be000800be007cda070069
:10a150000002be000404be002e019000be0190006b
:10a160004e009000de00900058d907000002be00ab
:10a170000401be000800be00b4d907000002be0002
:10a180006e019000fe0190000400be0050d907004f
:10a190000002be000400be00f0d907000002be00ad
:10a1a00004027800040078004f04be000080fa002a
:10a1b000000006000200fa00000f78000000000016
:10a1c00001003700000000003438800062026200a5
:10a1d000e00f5200fbff3a001e02780004388800ae
:10a1e00004602600143888000080fa000000060091
:10a1f0000400fa00008fbe000000000001003700dc
:10a20000000000003438800061026200e00f52005c
:10a21000fbff32001e02be00040278006438880092
:10a220001e02be0004027800743888001e02be00c0
:10a2300004027800843888001e02be000402780000
:10a24000943888000080fa00000006000800fa0038
:10a25000000f780011079800220798003307980034
:10a2600000000000010037000000000034388000ca
:10a2700062026200e00f5200fbff3a009e02900073
:10a280000405200004aab900040278001e0242005e
:10a29000043888001e0278006120b8001e02900079
:10a2a000050020000605200006abb9000603780073
:10a2b0006021b9008203780007034300840278001c
:10a2c00004052000042ab800050343008602780034
:10a2d0000002420081824a00402ade0084027800a7
:10a2e00004302600050272001438880000000000c7
:10a2f0000100370000000000343880006202620074
:10a30000e00f5200fbff3a002e029000cc22dd004d
:10a310003e02900005027200043888002e02900070
:10a32000c422de00044026000502720014388800b2
:10a3300000000000010037000000000034388000f9
:10a3400062026200e00f5200fbff3a0004062000a8
:10a350000438880004702600143888000080fa0051
:10a36000000006000800fa00008fbe0022079800d7
:10a3700033079800000000000100370000000000d3
:10a380003438800062026200e00f5200fbff3a00a6
:10a390002e029000be02900004027800043888006b
:10a3a0000420260014388800000000000100370057
:10a3b000000000003438800062026200e00f5200aa
:10a3c000fbff3a001e02be00040278000438880039
:10a3d0000430260014388800000000000100370017
:10a3e000000000003438800062026200e00f52007a
:10a3f000fbff3a00041e2f000438880004402600aa
:10a400001438880000000000010037000000000040
:10a410003438800062026200e00f5200fbff3a0015
:10a42000040e2000043888000470260014388800c8
:10a430000080fa00000006002e00fa00881f780055
:10a44000700f9800011798001217980023179800b2
:10a45000341798004517980056179800671798000a
:10a460007e0990008e1190003e109000ce1090005a
:10a4700096d807000002be0005f0a100140798005e
:10a48000250798001e119000ae1190005e109000fc
:10a49000ee1090008dd807000002be0005f0a1006c
:10a4a000340798004507980018c0b3003e0190009b
:10a4b000ce0190001e009000ae00900025d907004c
:10a4c00000027800e00f520001003c000044eb0065
:10a4d000e04f5400030032001e029000ae029000d4
:10a4e000020037003e029000ce0290005407980010
:10a4f000650798007e0990008e1190003e10900034
:10a50000ce10900071d807000002be005e019000de
:10a51000ee0190000400be00ccd807000002be008f
:10a5200074079800050f98001e119000ae1190005e
:10a530005e109000ee10900064d807000002be008c
:10a540005e019000ee0190000400be00bfd807003d
:10a550000002be00140f9800250f98000002eb00c7
:10a56000040f7800390037007e0190008e099000ba
:10a570007e0890008e10900055d807000002be00a3
:10a58000740f9800051798007e0890008e109000b8
:10a59000f2d807000002be0004027800cfa2de005d
:10a5a000340f9800450f98001e099000ae099000e6
:10a5b0001e109000ae10900045d807000002be00ab
:10a5c00014179800251798001e109000ae109000e8
:10a5d000e2d807000002be0004027800cfa2de002d
:10a5e000540f9800650f98003e0b9000ce0b900022
:10a5f000f404200005002000840f5300858f5b00c9
:10a6000011003e005e0b9000ee0b9000f41d200048
:10a6100005002000840f5300858f5b000a003e0078
:10a6200030002000e3fe07005e0a9000ee0a900072
:10a6300066024200e0824a000401be003e0890002b
:10a64000ce089000f9f407001e0fe8005e009000ad
:10a65000ee009000c1d807000002be00040278009e
:10a660009e0f5200c0ff3e004f0478000080fa00a9
:10a67000000006001000fa00008fbe0022079800bc
:10a68000330798004407980055079800660798001c
:10a69000770798000080fa00000006000000fa002a
:10a6a0000000000001003700000000003438800086
:10a6b00062026200e00f5200fbff3a000000eb0074
:10a6c000bcfe0700031e2000f20420008000eb0007
:10a6d0000000eb00ddfe07000080fa00000006002d
:10a6e0000000fa000000eb00b2fe0700031e20008d
:10a6f000120020008000eb00f0042000d3fe0700d1
:10a700000080fa00000006000200fa00000f780046
:10a710001e007800a7fe0700031e20001200200084
:10a720008000eb000000eb00c8fe0700031e2000c5
:10a73000120020008000eb00e0042000c3fe0700b0
:10a7400084cb2000144278000482fb00840178004e
:10a75000e20420008000eb000000eb00bbfe0700dd
:10a7600084cb2000144278008482fb0084cb20003c
:10a77000144278000482fb00061e200004025300ed
:10a7800085017800e2042000840078000000eb00de
:10a79000aefe07000080fa00000006000000fa008c
:10a7a0000000eb0083fe0700e46580008401780070
:10a7b000f20420008000eb000000eb00a3fe070085
:10a7c000e5658000e4658000061e20000402530059
:10a7d00085017800f2042000840078000000eb007e
:10a7e0009afe0700e565800034062000848f520041
:10a7f00003003e00e46580000482e800e465880010
:10a800000080fa00000006000000fa0031e7a8000e
:10a810000080fa00000006000400fa00004f7800f3
:10a82000110798009e42780004732000054a7800c2
:10a830003107a8001e029000943988000000000033
:10a84000010037000000000085398000040024006a
:10a8500004826200e00f5200faff3a003107a900bb
:10a860000080fa00000006000a00fa000002eb0077
:10a870001407980000c2eb004447980000c2eb00a8
:10a88000544798000042eb00044f7800280037003e
:10a8900068004700e703470066034700de42900078
:10a8a0004e4290009e4178000001780087007800b9
:10a8b00006007800a00007000e4a90000483fb0009
:10a8c0007e4290008482fb006e4290000482fb0076
:10a8d0000601780085007800040078003200070047
:10a8e00000027800140798001e427800e04f5200e2
:10a8f00004003a008000eb001e407800c6ff07000d
:10a900000a0037001e427800e24f420004003a007d
:10a910008080eb001e407800bfff07000300370077
:10a920009e0090001e407800bbff07001e4fe8000d
:10a930001e427800e14f4200d5ff3a000080fa0045
:10a94000000006000a00fa00000f780011079800c6
:10a950002207980033079800440798001e029000d1
:10a960009e0212004e0390003e029000040253002b
:10a9700004aab900840278002e0390001e02900001
:10a9800004025300110009008482d80000027800fc
:10a99000840278003e0290000482420004007800a5
:10a9a0000080fa00000006000600fa00000f7800a0
:10a9b0001107980022079800f40120008001eb00a5
:10a9c000f20f20008000eb001e007800ddff070082
:10a9d00000027800040f7800f40320008001eb00ef
:10a9e000f20f20008000eb001e009000d5ff070052
:10a9f0000002780014079800f40120008001eb00a9
:10aa0000f20f20008000eb002e009000cdff070029
:10aa100000027800240798001e0278004b22dd0017
:10aa2000040f78001e029000c522dd00047e200085
:10aa300004826200140798002e0290007f026200d8
:10aa4000240798001e0290009e0272002e029000c1
:10aa500005027200040078000080fa000000060081
:10aa60000400fa00004f7800114798002247980030
:10aa70001e4278008482fb00740020008001eb00fd
:10aa8000f20f20008000eb0005007800adff07000a
:10aa900000027800044f78001e4290008482fb0080
:10aaa000740020008001eb00f20f20008000eb001a
:10aab00005007800a3ff0700000278001447980003
:10aac0002e4290008482fb00340020008001eb00c5
:10aad000f20f20008000eb000500780099ff0700ce
:10aae00000027800244798009e4278000582fb000f
:10aaf0004522dd00044f78001e4290000482fb00d6
:10ab00004222dd00044278007c4262001447980033
:10ab10002e42900063426200244798001e4290003b
:10ab20009e4272002e42900004c2720004407800df
:10ab30000080fa00000006001400fa005007980098
:10ab400061079800720798000357980014579800ff
:10ab5000255798001e529000e04f52000c003a001a
:10ab60007e0290002e509000004a78007e029000f5
:10ab7000944278006e029000054a78006e029000c0
:10ab8000944278005e029000054a780091003700f8
:10ab90000e5290008482fb00b402200011000900d4
:10aba0008482d80000027800044278000482fb000e
:10abb000040f78000e5290000483fb009e02780080
:10abc000b402200004aab900040278000402530071
:10abd0006622b90004027800140798002e529000f3
:10abe0008482fb001e5290000482fb00f60f2000be
:10abf0000402530004aab9000402780048a2de004f
:10ac0000240798002e5290000483fb001e529000ef
:10ac10008482fb001e02900004aab900040278009e
:10ac20004822de00f50f20000482520004b2b90071
:10ac3000040278004822de00340798002e5290006b
:10ac40000483fb001e5290008482fb00f70f20005b
:10ac50001e0290000482530004aab9000402780086
:10ac60004822de00f50f20000482520004b2b90031
:10ac7000040278004822de00440798001e02780093
:10ac8000050020004600200007002000860f52002b
:10ac9000878f5a0042003e00046001000400370024
:10aca0000f0037001a00370025003700300037004a
:10acb0005e029000ae529000054a78004e0290006d
:10acc000844278006e029000054a78002e029000bf
:10acd000844278007e029000054a78003c003700ec
:10ace0003e029000844278005e029000054a78009f
:10acf0006e0290002e509000004a78002e029000c4
:10ad0000844278007e029000054a780030003700c7
:10ad10002e029000844278005e029000054a78007e
:10ad20006e029000ae509000014a78004e029000f2
:10ad3000844278007e029000054a780024003700a3
:10ad40002e029000844278005e029000054a78004e
:10ad50003e029000844278006e029000054a78001e
:10ad60007e029000ae529000054a7800180037002d
:10ad70004e029000844278005e029000054a7800fe
:10ad80002e029000844278006e029000054a7800fe
:10ad90007e0290002e509000004a78000c00370090
:10ada0005e029000ae509000014a78002e029000a2
:10adb000844278006e029000054a78003e029000be
:10adc000844278007e029000054a7800000000006e
:10add000000000000080fa00000006000c00fa00ed
:10ade000881f78008a9fbe008c9fbe0004508000a0
:10adf00022a02000030020006123b9006c3ab900b2
:10ae0000040078006032b9000402780004004000b9
:10ae100086027800c4002000042ab8000500400023
:10ae200080027800848fd2008582d20004027800ec
:10ae300004f0a100100020008200d0000403d00024
:10ae4000068240004220a800858249004200a900f5
:10ae50004220ae004200a8000482d300a601800078
:10ae60008503780004027800a7018800000a7800b2
:10ae7000a60188000850800097d8070000027800db
:10ae8000cfa2de00e2042000030020000400be0088
:10ae9000cad707000002be000401780027a02000e6
:10aea000070f780000002000100798006142b900e9
:10aeb0006c2bb900060378006020b900800378008d
:10aec0000703430084027800c4002000042ab8006d
:10aed000050343008602780062024200e0824a00d5
:10aee000848fd2008582d2000402780004f0a10091
:10aef0001e03be000600d0008400d0000102400006
:10af00004220a80085824b004200a9004220ae00ea
:10af10004200a8000482d300a601800085037800c7
:10af200004027800a7018800020a7800a6018800c0
:10af30000850800068d8070000027800cfa2de0029
:10af4000921d2000030020000400be009bd70700d4
:10af50000002be00040278000401e80023a02000e3
:10af60002307980004002000340798006142b900cc
:10af70006c2bb900060378006020b90080037800cc
:10af80000703430084027800c4002000042ab800ac
:10af9000050343008602780064024200e0824a0012
:10afa000848fd2008582d2000402780004f0a100d0
:10afb0002e039000be0390000600d0008400d00055
:10afc000010240004220a80085824b004200a900f7
:10afd0004220ae004200a8000482d300a6018000f7
:10afe0008503780004027800a7018800020a78002f
:10aff000a60188000850800037d8070000027800ba
:10b0000025002000110009000502d8000102780087
:10b010000402e8000401780023a020004307980000
:10b0200004002000540798006142b9006c2bb9005d
:10b03000060378006020b90080037800070343000e
:10b0400084027800c4002000042ab80005034300ed
:10b050008602780066024200e0824a00848fd200b5
:10b060008582d2000402780004f0a1004e03900013
:10b07000de0390000600d0008400d00001024000f2
:10b080004220a80085824b004200a9004220ae0069
:10b090004200a8000482d300a60180008503780046
:10b0a00004027800a7018800020a7800a60188003f
:10b0b000045080002ca020000d002000cfa2de0054
:10b0c0006c2bb900060378006020b900800378007b
:10b0d0000703430084027800c4002000042ab8005b
:10b0e000050343008602780068024200e0824a00bd
:10b0f000848fd2008582d2000402780004f0a1007f
:10b100008003eb008c01d0000403d00006824100d4
:10b110004220a80085824e004200a9004220ae00d5
:10b120004200a8000482d300a60180000500780038
:10b1300004027800a0018800070a7800a6018800b0
:10b1400008508000e4d7070000027800040178006e
:10b150002aa020000b0020006142b9006c2bb9002e
:10b16000060378006020b9008003780007034300dd
:10b1700084027800c4002000042ab80005034300bc
:10b18000860278006a024200e0824a00848fd20080
:10b190008582d2000402780004f0a1008a03d00066
:10b1a0000400d000008243004220a80085824d00a8
:10b1b0004200a9004220ae004200a8000482d30051
:10b1c000a60180008503780004027800a7018800aa
:10b1d000020a7800a6018800045080000402e800fa
:10b1e000045088004f06be004f05be004f04780093
:10b1f0000080fa00000006000200fa00889fbe00ee
:10b200008a9fbe008c9fbe004487a8003d3a800004
:10b21000fc1f20008c8666000ca028000d0676001e
:10b220003c3a88000ac025000b0020000a0578007f
:10b23000ca38880008c0250009002000404cde0004
:10b2400088047800f80f200008846400d83888004b
:10b2500002c0250003002000020178006238880047
:10b2600000c02500010020004008de0080007800ba
:10b27000f00f2000008060007038880006c02500b4
:10b2800007002000060378008638880004c02500e7
:10b2900005002000402ade0084027800f40f200020
:10b2a000048262009438880004052000a4388800d5
:10b2b000041e2000b4388800243980000400a00057
:10b2c0000410a1000420a100243988000082eb00b2
:10b2d000f4398800a538800004802f008482620041
:10b2e0000405200005027200a4388800a5388000fb
:10b2f000f47f200084826200f47f200004826200d8
:10b30000e638800005802f00850263000502720088
:10b31000e4388800b538800004802f008482620001
:10b32000041e200005027200b4388800b538800081
:10b33000f47f200084826200f47f20000482620097
:10b34000f638800005802f00850263000502720038
:10b35000f43888000539800004802f008482620060
:10b36000040a2000050272000439880015398000a3
:10b3700004802f00848262002421200005027200d4
:10b380001439880026e7a9002647a90026c7a90086
:10b390002627a8002607a80026a7a9002687a90017
:10b3a00094c1b30004437800f5722000864a780007
:10b3b000f472200014427800044378009572200053
:10b3c000864a780004c5b30004437800e572200083
:10b3d000864a7800e4722000144278000443780022
:10b3e00085722000864a7800a4c0b3000443780028
:10b3f000c5722000864a780004c2b3000443780076
:10b40000a5722000864a780054c0b3000443780037
:10b41000d5722000864a780004c1b3000443780046
:10b42000b5722000864a78002667a9002727a80061
:10b430002707a8000002eb00040f78000100370086
:10b440001e0fe800850020001e02780004aade001e
:10b45000e10f5200faff3c001e027800044278001f
:10b46000674262000482fb00670262004522dd0041
:10b4700026388000f5f12f00850263000502720076
:10b4800024388800243880004522de0067426200ac
:10b490000482fb00670262004522dd00263980003d
:10b4a000f5f12f008502630005027200243988003f
:10b4b00005e7a80000e8230001002000690107005b
:10b4c0004f06be004f05be004f04be000080fa00cc
:10b4d000000006000400fa00008fbe001e02be003d
:10b4e00004027800843888001e02be00040278003e
:10b4f000943888001e02be0004027800c438880018
:10b500001e02be0004027800d43888000080fa00d1
:10b51000000006000000fa000000000001003700f3
:10b5200000000000343880006102620004f0a700cf
:10b530000402ea000402e9004f22de0035388000f0
:10b54000c72ade00e1c262008582fb0084827200ad
:10b55000343880004622de00614262000482fb0033
:10b5600085027200343880004522de0061426200ac
:10b570000482fb0005027200e00f5200e8ff3a006f
:10b58000140020003465880000000000010037002e
:10b590000000000034658000e00f5200fcff3a001c
:10b5a0000080fa00000006000000fa0000c025003c
:10b5b0000100200054658000cfa2de000660290053
:10b5c00006abb900060378006021b9008203780059
:10b5d000070343008402780004602900042ab800ad
:10b5e0000503430086027800848fd2008582d20052
:10b5f0000402780004f0a1000003d0008403d0000e
:10b60000070243004220a800858248004200a900aa
:10b610004220ae004200a8000482d3000400be0015
:10b62000f3fa07005465800004f0a7000402ea0062
:10b630000402e9004f22de005465880017fc070071
:10b640000080fa00000006003600f800809fbe006f
:10b65000829fbe00849fbe00869fbe003200f8001d
:10b6600000202000900188000000fa00543880007b
:10b6700070026200e00f5200300032000002eb0066
:10b6800064658800746580000402e80074658800c1
:10b6900034658000e00f52002400320000c0250015
:10b6a0000100200004668000cfa2de0006602900b1
:10b6b00006abb900060378006021b9008203780068
:10b6c000070343008402780004602900042ab800bc
:10b6d0000503430086027800848fd2008582d20061
:10b6e0000402780004f0a1000003d0008403d0001d
:10b6f000070243004220a800858248004200a900ba
:10b700004220ae004200a8000482d3000400be0024
:10b7100070ff07000466800004f0a7000402ea003e
:10b720000402e9004f22de00046688000002eb00fc
:10b73000346588000a87a900080037005438800063
:10b7400068026200e00f520004003200646580006d
:10b750000402e800646588000a67a9009080a900d7
:10b760000080fa003200f9004f03be004f02be0015
:10b770004f01be004f00be003600f9000040060039
:10b780000000fa0000000000010037000000000087
:10b790003438800062026200e00f5200fbff3a0082
:10b7a0000082eb000438880004002500143888006b
:10b7b0000000000000000000010037000000000051
:10b7c0003438800062026200e00f5200fbff3a0052
:10b7d0000002eb00043888000410250014388800ab
:10b7e0000000000000000000010037000000000021
:10b7f0003438800062026200e00f5200fbff3a0022
:10b80000c42a250004388800042025001438880044
:10b8100000000000000000000100370000000000f0
:10b820003438800062026200e00f5200fbff3a00f1
:10b830000002eb00043888000480250014388800da
:10b8400000000000000000000100370000000000c0
:10b850003438800062026200e00f5200fbff3a00c1
:10b86000041e2000043888005490250014388800f5
:10b87000000000000080fa00000006000800fa0046
:10b88000100798002107980032079800f46580009f
:10b89000840278003e029000848f52000200310042
:10b8a000f4658000340798001e0090002ad6070037
:10b8b0000002be00040278006622b900040278008b
:10b8c000f504200004825200040f78009e027800e4
:10b8d0002e029000848f5200030031001e02780077
:10b8e0002407980003003700000000000100370023
:10b8f000000000003438800062026200e00f520055
:10b90000fbff3a002e029000cc22dd003e029000a8
:10b9100005027200043888002e029000c422de0066
:10b9200004a0250005027200143888000000000001
:10b930001100370000000000010037000000000087
:10b940003438800062026200e00f5200f9ff3a00d2
:10b950001e029000144278000402fb0004388800a4
:10b960000430250014388800000000001e029000fa
:10b970000402e800140798001e02900014427800a8
:10b98000e04f5200edff3a000080fa000000060090
:10b990000000fa000002eb00140888002405800073
:10b9a00004c0a00004d0a10004e0a0002405880089
:10b9b00005e1a8008460a9009460a80094d021004b
:10b9c000640888003405800004c0a10004d0a000f1
:10b9d00004e0a0003405880084e0a90004032800e6
:10b9e0008408880094e0a8000080fa0000000600a7
:10b9f000849fbe00861f78003200f80004202000db
:10ba0000940188000000fa00d46580000500200041
:10ba10000402420085824a00e6be2000060242007f
:10ba20001402780014088800d46580000402e8003d
:10ba3000d4658800d565800004042000848f5200fe
:10ba400002003a000002eb00d465880084e0a900ff
:10ba50000080fa003200f9004f0378004f02be0068
:04ba6000004006009c
:020000040000fa
:10ba6400f03fb1000180b10006003500ee0309008b
:10ba740000000000403fb1000180b100fbff3d0029
:10ba84001000b000203fb000020035000080090023
:08ba94000000000000000600a4
:020000040000fa
:020000040005f5
:0457f400ffec0000c6
:020000040000fa
:020000040005f5
:0457f800be9b000054
:020000040000fa
:020000040005f5
:0457fc007f3f0000eb
:00000001FF
